:100000000C9412030C942F030C942F030C942F03C5
:100010000C942F030C942F030C942F030C942F0398
:100020000C942F030C942F030C94502E0C94222F1D
:100030000C9426290C942F030C942F030C942F035B
:100040000C942F030C942F030C942F030C942F0368
:100050000C942F030C94CA290C942F030C942F0397
:100060000C942F030C942F030C942F030C942F0348
:100070000C942F030C942F030C942F030C942F0338
:100080000C942F030C942F030C942F030C942F0328
:100090000C940D270C942F030C942F030C942F0316
:1000A0000C942F030C942F030C942F03CB06CB0638
:1000B000F706F7065F077D0795089508880721086A
:1000C000320832088F2FB62FAE30B62FAE30023046
:1000D0002530AE307C308B3007634236B79BD8A7D3
:1000E0001A39685618AEBAAB558C1D3CB7CC57635D
:1000F000BD6DEDFD753EF6177231BF000000803F0B
:1001000005A84CCDB2D44EB93836A9020C50B991DD
:100110008688083CA6AAAA2ABE000000803F4D653A
:10012000736F6E206D6163726F20776F726B696E93
:100130006700290014001A000800150017002B00A2
:10014000E00004001600070009000A00E200E100D8
:100150001D001B00060019000500E3000000000060
:100160000000000001512C0000002A0013001200C2
:100170000C0018001C003100280033000F000E0096
:100180000D000B0035003400380037003600100039
:1001900011000500000000000000000002512C00CA
:1001A000000035021E021F022002210222022B0043
:1001B000E0003A003B003C003D003E003F00E10013
:1001C0002D022E022F0230023102E3000000000057
:1001D0000000000001512C000000CA5C270226022A
:1001E0002502240223023100CB5C45004400430079
:1001F000420041004000C45CA75D01004F00520076
:1002000051005000000000000000000003512C00CD
:10021000000035001E001F002000210022002B00DE
:10022000E0003A003B003C003D003E003F00E100A2
:100230002D002E002F0030003100E30000000000F0
:100240000000000003512C000000A9002700260038
:100250002500240023003100AA004500440043008B
:10026000420041004000AE00AB00AC004F00520025
:1002700051005000000000000000000002512C005E
:100280000000005C0100010001000100010001000C
:100290000100010001000100010001000100010056
:1002A0000100010001000100010001000000000048
:1002B0000000000001000100000001000100010039
:1002C0000100010001000100010001000100010026
:1002D0000100010001000100010001000100010016
:1002E000010001000000000000000000010001000A
:1002F000000000000000000000002A2B2800000081
:1003000000000000000000000000000000290000C4
:1003100000002C1E3420212224342627252E362DA1
:100320003738271E1F202122232425263333362E3B
:1003300037381F0405060708090A0B0C0D0E0F10AD
:100340001112131415161718191A1B1C1D2F3130F2
:10035000232D350405060708090A0B0C0D0E0F1096
:100360001112131415161718191A1B1C1D2F3130D2
:10037000354C0000000000000000000000000000FC
:10038000000000000000000000000000000000006D
:100390000000000000007E0F00D4FFFFFFC7000038
:1003A000007800047F3F1F643214643214783C1ECE
:1003B0001E140A05FFAA7F55400001010101010139
:1003C000010101020202020202020202030303030C
:1003D00003030303040404040404040505050505DC
:1003E000060606060607070707070808080809099A
:1003F00009090A0A0A0B0B0B0C0C0C0D0D0D0E0E45
:100400000E0F0F0F101011111112121313141415D7
:100410001516161717181819191A1A1B1B1C1D1D4B
:100420001E1E1F20202122222324242526262728A1
:1004300029292A2B2C2D2D2E2F30313232333435D1
:10044000363738393A3B3C3D3E3F404142434445D4
:10045000464748494A4C4D4E4F50515354555658B3
:10046000595A5B5D5E5F616264656668696B6C6D5D
:100470006F7072737577787A7B7D7E8082838587D3
:10048000888A8C8E8F91939596989A9C9EA0A2A311
:10049000A5A7A9ABADAFB1B3B5B7BABCBEC0C2C416
:1004A000C6C9CBCDCFD1D4D6D8DBDDDFE2E4E7E9D6
:1004B000EBEEF0F3F5F8FAFDFF0C034D0065007369
:1004C000006F006E00000014034C007500630069AB
:1004D0000061006E006F0020004D00000004030961
:1004E0000409023B00020100A0FA09040000010314
:1004F00001010009211101000122400007058103CB
:100500000800010904010001030000000921110194
:10051000000122B60007058203200001120100023B
:1005200000000008EDFE00000100010200010501CD
:100530000902A10185020901A10005091901290883
:100540001500250195087501810205010930093161
:100550001581257F95027508810609381581257F4B
:10056000950175088106050C0A38021581257F95CD
:100570000175088106C0C005010980A10185031924
:10058000012AB700150126B700950175108100C03A
:10059000050C0901A101850419012AA002150126F3
:1005A000A002950175108100C005010906A1018511
:1005B00006050719E029E715002501950875018151
:1005C000020507190029EF1500250195F075018135
:1005D0000205081901290595057501910295017516
:1005E000039101C005010906A101050719E029E7EA
:1005F0001500250195087501810295017508810195
:100600000507190029FF150026FF009506750881CA
:1006100000050819012905950575019102950175D7
:10062000039101C011241FBECFEFDAE0DEBFCDBFC2
:1006300011E0A0E0B1E0EAE8FAE602C005900D9210
:10064000AA3EB107D9F723E0AAEEB1E001C01D929E
:10065000A437B207E1F70E9439180C9443350C9483
:100660000000873A9D4541F4FB018281882321F0F7
:100670008EE191E00E94DA0481E0089581E008951E
:100680000C94310308950C9442031F93CF93DF938E
:1006900000D000D01F92CDB7DEB749835A836B8359
:1006A0003091ED0189819A81311114C0662359F08E
:1006B000222349F00E94D20A182F682F89819A813B
:1006C0000E947B0A03C00E94A60A182F69817A81C2
:1006D000812F04C00E94D20A69817A810F900F9005
:1006E0000F900F900F90DF91CF911F910C94FF11FD
:1006F000FC01262F408151816281738184810C9499
:10070000450381E00895CF93DF93EC0160E00E9400
:100710007803BE01DF91CF910C9443030C948C13AA
:100720000C94881308950E9425090E9492032FEFCC
:1007300084E39CE0215080409040E1F700C000003D
:100740000C94F0290F931F93CF93DF938C0161E0FA
:100750000E947803EC01B8010E944003882309F449
:1007600044C0B801CE010E943B258823F1F1B801B5
:10077000CE010E944F238823C1F1B801CE010E940F
:100780009724882391F1B801CE010E943D2288234D
:1007900061F1F8018281882309F1CB358DE5D80715
:1007A000C1F050F4C115FCE5DF0781F0CF3DDC4519
:1007B000A9F40E94091019C0CC35EDE5DE0761F0FF
:1007C000CD35DD4559F40E944C0F08C00E949303BB
:1007D0000CC00E94550F02C00E94580FC801DF9143
:1007E000CF911F910F910C943E0380E0DF91CF9148
:1007F0001F910F9108950E9409290E94EE040C9404
:10080000E7200E94F1040E94A3200C940F29DF929C
:10081000EF92FF920F931F93CF93DF93E82FF0E0B7
:10082000EE50FD4FD490282F26952695269530E042
:10083000F901EE56FC4F0491877010E0082E02C0BB
:10084000159507950A94E2F701701127F901EE5703
:10085000FC4FE490F12C082E02C0F594E7940A9422
:10086000E2F791E0E922FF24F901EE58FC4FC49130
:10087000D0E002C0D595C7958A95E2F7C170DD2713
:100880000115110519F081EE0E945005E114F104E3
:1008900019F086EE0E9450058D2D0E947906EF28F2
:1008A00019F086EE0E94FA05012B19F081EE0E94E4
:1008B000FA05CD2B51F08CE2DF91CF911F910F9172
:1008C000FF90EF90DF900C947906DF91CF911F910C
:1008D0000F91FF90EF90DF900895EF92FF920F93AA
:1008E0001F93CF93DF938C01F62E8AE0E82EF80158
:1008F0008491882309F457C0813009F042C0E8018F
:100900002196FE018491813031F42196FE0184917B
:100910000E94790639C0823039F4E8012296FE013E
:1009200084910E94500530C0833039F4E80122964A
:10093000FE0184910E94FA0527C0843029F5E80160
:100940002296FE01249180E090E030E020533109AE
:100950002A30310560F4E89EA001E99E500D112473
:10096000C901840F951F2196FE012491EECF0097B7
:1009700059F0EFE9FFE03197F1F700C0000001976F
:10098000F6CF0E940704E8018E010F5F1F4F8F2DE5
:10099000882309F4ACCFEFE9FFE03197F1F700C00D
:1009A00000008150F5CFDF91CF911F910F91FF9003
:1009B000EF90089560E00C946D0408950C94DD04AC
:1009C00081E008950C94E0040895CF93C82F0E940D
:1009D000DE048C2F0E94E204CF91089580E00C94F5
:1009E000E5040E94C7270C94E5040E94C727909154
:1009F000EC01891721F08093EC010C94E504089533
:100A0000CF93DF93CDB7DEB72B970FB6F894DEBF49
:100A10000FBECDBF4F83588769877A878B87611157
:100A20000E94980E9E012F5F3F4F86E0F9011192C0
:100A30008A95E9F785E0FE013796D90101900D927C
:100A40008A95E1F789819A814C815D81452B31F04E
:100A50009F3F31F491E08F3F19F403C091E001C052
:100A600090E090FF09C049815A816B817C818D8122
:100A70009E810E94B90D05C0C9010E9481038111A8
:100A8000F2CF2B960FB6F894DEBF0FBECDBFDF912D
:100A9000CF910895FC01808191810E94140B0895EB
:100AA000CF93882309F4A4C0C82F8238C1F40E94D0
:100AB000C72781FD9DC069E38091020190910301E8
:100AC0000E94C4280E94BA0E2FEF81EE94E02150BC
:100AD00080409040E1F700C0000069E319C083380E
:100AE00001F50E94C72780FD83C063E58091020164
:100AF000909103010E94C4280E94BA0E2FEF81EE4C
:100B000094E0215080409040E1F700C0000063E590
:100B100080910201909103010E94CF28CF910C9403
:100B2000BA0E8438C1F40E94C72782FD61C067E411
:100B300080910201909103010E94C4280E94BA0E84
:100B40002FEF81EE94E0215080409040E1F700C00B
:100B5000000067E4DDCF8CEF8C0F813AD0F46C2F6E
:100B600080910201909103010E944428882349F05A
:100B70006C2F80910201909103010E94CF280E9466
:100B8000BA0E6C2F80910201909103010E94C4283B
:100B9000C5CF80E28C0F883048F4C77081E001C077
:100BA000880FCA95EAF70E947B0EB8CFEBE5EC0FF1
:100BB000E33040F4F0E0ED57FE4F808190E0CF91BC
:100BC0000C940228E8E5EC0FE73150F4F0E0EE0F6A
:100BD000FF1FEB5AFE4F80819181CF910C94182812
:100BE000CD3E30F08C2F0E94BE18CF910C949019FE
:100BF000CF910895882309F464C0823879F40E9463
:100C0000C72781FF5EC069E38091020190910301D3
:100C10000E94C4280E94BA0E69E310C08338B1F460
:100C20000E94C72780FF4DC063E58091020190912B
:100C300003010E94C4280E94BA0E63E5809102015C
:100C4000909103010E94CF280C94BA0E843879F455
:100C50000E94C72782FF35C067E48091020190910E
:100C600003010E94C4280E94BA0E67E4E7CF9CEFFC
:100C7000980F913A10F4682FE1CF90E2980F9830D6
:100C800050F4877091E001C0990F8A95EAF7892F97
:100C90000E94810ED9CF9BE5980F933020F480E01D
:100CA00090E00C94022898E5980F973120F480E0AA
:100CB00090E00C9418288D3E20F00E9419190C9495
:100CC000901908951F93CF93DF93182FEB010E9483
:100CD0005005209741F08FE99FE00197F1F700C0A0
:100CE00000002197F6CF812FDF91CF911F910C94B7
:100CF000FA05893319F060E070E002C060E570E049
:100D00000C946206882321F00E947B0E0C94BA0E8C
:100D10000895882321F00E94810E0C94BA0E089544
:100D2000CF92DF92EF92FF920F931F93CF93DF93B7
:100D30007C01D62FC72FFC011281058102950F700F
:100D40000E94710E8823B9F01123A9F08C2F807FA7
:100D5000803421F080E28D0F883068F080911B0391
:100D600082FD09C082E00E941A0F0E94710E91E07C
:100D7000D82ED92601C0D12CCC2EC2948FE0C82207
:100D80008C2D90E08C30910508F0CFC1FC01EA5A1F
:100D9000FF4F0C9495348C2F807FCF70882311F0F7
:100DA000C295C07F112399F0CC2309F4AAC180E237
:100DB0008D0F883010F0D11104C08C2F0E947B0E53
:100DC00003C08C2F0E948B0E0E94BA0E9AC18D2FE9
:100DD0000E94FA05CC2309F4A8C180E28D0F883067
:100DE00038F1DD2329F18C2F0E94910E24C08C2F25
:100DF000807FCF70803211F0C295C07FDD2319F063
:100E0000D130A1F13DC080911B0382FF17C0112397
:100E100049F0CC2329F08C2F0E947B0E0E94BA0E41
:100E200080E070C180E00E94FA05CC2309F47DC106
:100E30008C2F0E94810E0E94BA0E77C1112371F08F
:100E4000002341F0013031F40E949B0E8C2B0E9454
:100E5000A30E6BC10E949B0E8C2B1DC0002319F0AA
:100E6000013009F462C10E94B00E25C0112321F0A7
:100E7000063008F05AC10EC0053008F056C11BC03C
:100E8000112361F0002331F0F701858180FF39C122
:100E90008F7085838C2F0E94820647C1002359F0F2
:100EA000D93309F03FC1FFEF07EE13E0F1500040E6
:100EB0001040E1F735C18C2F0E94890636C18C2F76
:100EC00086958695837019F0813061F02EC11123CB
:100ED00021F08D2F9C2F937002C080E090E00E9443
:100EE00002282BC1112321F08D2F9C2F937002C05B
:100EF00080E090E00E94182820C18D2F112319F066
:100F00000E94BE1802C00E9419190E94901915C1B2
:100F10008C2F837009F047C011110BC12D2F229522
:100F200026952770220F220F6D2F6F70862F90E06D
:100F3000A0E0B0E0022E04C0880F991FAA1FBB1FBB
:100F40000A94D2F7D4FF10C04FE050E060E070E0A8
:100F500004C0440F551F661F771F2A95D2F740958E
:100F600050956095709503C040E050E0BA01C69579
:100F7000C695C3708A019B01082B192B2A2B3B2B8A
:100F8000C901B801C23049F058F4C13019F00E94CB
:100F90009109CFC00E947F09CCC00E94A309C9C09B
:100FA0000E947D09C6C0112319F08C2F817001C0E9
:100FB0008695882309F4BDC02D2F2295269527708C
:100FC000220F220F6D2F6F70862F90E0A0E0B0E00F
:100FD000022E04C0880F991FAA1FBB1F0A94D2F7C4
:100FE000D4FF10C04FE050E060E070E004C0440F58
:100FF000551F661F771F2A95D2F74095509560952B
:10100000709503C040E050E0BA01C695C695C37024
:101010008A019B01082B192B2A2B3B2BC901B801F4
:10102000C23049F058F4C13019F00E94560A81C00C
:101030000E94440A7EC00E94680A7BC00E94B709D1
:1010400078C0CF70112339F08C2F0E94DD098D2FCD
:101050000E9482066EC08D2F0E9489068C2F0E94EE
:10106000FE0967C0D23F21F128F4D03F41F0D13FC3
:10107000C1F043C0D33F19F1D43F79F03EC01123F2
:1010800041F0053008F051C08C2F8F710E94230A67
:101090004CC0063008F049C0F7CF80911B0382FF97
:1010A00018C0112339F08C2F8F710E94DD093DC0CB
:1010B0001123C9F38C2F8F710E94FE0936C01123B2
:1010C00029F08C2F8F710E94C8092FC00E94C3097C
:1010D0002CC0112349F0CF718C2F0E94DD0963E0F1
:1010E0008C2F0E94FF0E21C081E00E941A0F023057
:1010F000E0F082E00E941A0F18C0112331F00023A3
:1011000091F28D2F0E94500510C0002399F2D9331F
:1011100049F41FEF27EE33E0115020403040E1F753
:1011200000C000008D2F0E94FA0588EF8C0D8430DE
:1011300020F40E94C7270E94E504DD20C9F00E9428
:101140006D0E80FD15C0F70112820E94670E0E948D
:10115000DD09C7010E94D9080E94670EDF91CF9177
:101160001F910F91FF90EF90DF90CF900C94FE09AC
:10117000DF91CF911F910F91FF90EF90DF90CF9073
:1011800008950F931F93CF93DF93EC0168817981CA
:101190008A810E941F0B8C010E947A0A0E946B09AF
:1011A000B801CE010E949006DF91CF911F910F915F
:1011B0000895CF93DF93EC01988189812B813C8145
:1011C000232B31F08F3F31F481E09F3F19F403C0AE
:1011D00081E001C080E080FD1DC0CE010E94A2031D
:1011E000811110C00E94710E8823A1F08A8188238A
:1011F00089F080911B0382FD0DC082E0DF91CF91C9
:101200000C941A0FCE010E94C108CE01DF91CF913C
:101210000C948303DF91CF91089580E090E00E94C9
:10122000022880E090E00E9418280E94980E0E94F8
:10123000BA0E0E94C11A0C949019809102019091EB
:1012400003010E94DA280C940D090E94880E0C9468
:101250001D0992959F70963079F010F4925001C05C
:101260009A50923068F4803F69F018F4883E40F458
:1012700009C0843F29F406C0883E20F0813F11F068
:1012800080E0089581E00895FC01808191810E94B1
:10129000140B0E9429090895CF93DF9300D000D04A
:1012A0001F92CDB7DEB70F900F900F900F900F9059
:1012B000DF91CF910895CF93DF9300D000D000D07D
:1012C000CDB7DEB726960FB6F894DEBF0FBECDBF02
:1012D000DF91CF910895089508950C946C090C94B2
:1012E0006D090E946F096093150270931602809336
:1012F0001702909318020C940D090C9471090F9326
:101300001F9300911502109116022091170230913F
:101310001802602B712B822B932B1F910F910C9431
:1013200071090F931F9300911502109116022091DD
:1013300017023091180260237123822393231F9197
:101340000F910C9471090F931F9300911502109146
:101350001602209117023091180260277127822708
:1013600093271F910F910C9471090C946C090E94A2
:10137000B509609311027093120280931302909347
:1013800014020C940D0960E070E0CB010C94B709D5
:101390000F931F9341E050E060E070E08A019B01F1
:1013A00004C0000F111F221F331F8A95D2F7C901F5
:1013B000B8011F910F910C94B7090F931F9341E04F
:1013C00050E060E070E004C0440F551F661F771FB7
:1013D0008A95D2F78091110290911202A091130286
:1013E000B09114028A019B01082B192B2A2B3B2B4D
:1013F000C901B8011F910F910C94B7090F931F9366
:1014000041E050E060E070E004C0440F551F661FEB
:10141000771F8A95D2F74095509560957095809189
:10142000110290911202A0911302B09114028A014C
:101430009B01082319232A233B23C901B8011F91CB
:101440000F910C94B7090F931F9341E050E060E0B7
:1014500070E004C0440F551F661F771F8A95D2F7AE
:101460008091110290911202A0911302B091140286
:101470008A019B01082719272A273B27C901B801A0
:101480001F910F910C94B7090F931F9300911102B4
:10149000109112022091130230911402602B712BD3
:1014A000822B932B1F910F910C94B7090F931F93CD
:1014B0000091110210911202209113023091140236
:1014C00060237123822393231F910F910C94B709FA
:1014D0000F931F9300911102109112022091130299
:1014E0003091140260277127822793271F910F9153
:1014F0000C94B709089527E0929F800D1124E82FDE
:10150000E695E695E695877051E001C0550F8A95FE
:10151000EAF785E0E89FF0011124E251FE4F20E058
:1015200030E070E04081CB01022E02C09695879595
:101530000A94E2F78170819584278523842781931B
:101540002F5F3F4F2530310569F7089527E0929FBF
:10155000800D1124682F669566956695982F977073
:1015600085E0689FB001112440E050E080E0FB017D
:10157000E40FF51FE251FE4F208130E0092E02C03A
:10158000369527950A94E2F721703327042E01C07F
:10159000220F0A94EAF7822B4F5F5F4F45305105C7
:1015A00031F70895BF92CF92DF92EF92FF920F939F
:1015B0001F93CF93DF938C01C0901102D090120241
:1015C000E0901302F090140280911502909116029F
:1015D000A0911702B0911802C82AD92AEA2AFB2A38
:1015E000CFE1D0E0D701C6010C2E04C0B695A79577
:1015F000979587950A94D2F780FD04C0219790F7BC
:10160000B12C07C0BC2EB8018C2F0E94121201977A
:10161000A9F38B2DDF91CF911F910F91FF90EF9048
:10162000DF90CF90BF900895CF93DF93EC010E949D
:10163000D20ABE010E941212DF91CF9108951F932A
:10164000CF93DF93EB019091ED01992321F0CB0132
:101650000E94140B13C0882349F0CB010E94D20AC8
:10166000182F682FCE010E947B0A04C0CB010E9474
:10167000A60A182FBE01812F0E941212DF91CF916E
:101680001F9108951F93CF93DF93C091190216E025
:1016900080911A02C81799F0D0E01C9FF0011D9F9D
:1016A000F00D1124E55EFD4F40815181628173810F
:1016B000848195810E945B092196C770E9CFDF91F3
:1016C000CF911F91089540914B0250914C0260912F
:1016D0004D0270914E0280914F02909150020C94F5
:1016E0005B09EF92FF920F931F93CF93DF9380914B
:1016F000500282958F7009F065C080914D02882359
:1017000009F460C080911902F0901A0210914B0206
:1017100000914C0260914E0270914F0291E01F3F88
:1017200009F090E0C0910001D0910101292F96E0CD
:10173000E92E8F1509F446C06115710521F00F3FA0
:1017400021F030E003C031E001C0322F90E030FDE5
:1017500036C0E89EF001E99EF00D1124DF01A55E80
:10176000BD4F11963C911197301329C03C91311314
:1017700026C012963C911297311121C013964D91BB
:101780005C911497461B570B4C175D07C0F4809172
:1017900050028F70806180935002E05EFD4F808127
:1017A0008F70806180838BE492E00E94D908DF9182
:1017B000CF911F910F91FF90EF900C94420B0196E7
:1017C0008770B7CFDF91CF911F910F91FF90EF906E
:1017D00008959F92AF92BF92CF92DF92EF92FF92C5
:1017E0000F931F93CF93DF93CDB7DEB761970FB6FB
:1017F000F894DEBF0FBECDBF8C0185E0F801DE019D
:101800001D9601900D928A95E1F7D8011296EC9001
:1018100090914B02E0914C0220914E0230914F0288
:101820002115310531F0EF3F31F481E09F3F19F48C
:1018300003C081E001C080E0B82FB1709B2E80FD15
:1018400047C1D8014C9111965C9111971396AD90B8
:10185000BC9014978BE4C82E82E0D82EF0904D02F5
:10186000B501621B730B2091000130910101FF2033
:1018700009F4D9C0809150026217730708F095C02F
:10188000282F207F09F052C05E1313C0491311C0E6
:10189000FE2CE1100EC08F708061809350020E9478
:1018A000630BC6010E94D90880915002F80185831C
:1018B0004DC1AB2831F05F3F31F481E04F3F19F467
:1018C00003C081E001C080E080FD03C081E08E257F
:1018D00002C080E090E0F82FF170FF2E80FF1CC066
:1018E0008091190220911A0236E0821709F40BC187
:1018F00090E0389FF001399FF00D1124E55EFD4F17
:101900006181561306C06081461303C06281E612EE
:1019100003C001968770E9CFFE2CEE2009F416C1B2
:101920008091500281608093500254C05E1306C0C3
:10193000491304C0E11002C0F80199C0C8010E9417
:101940004409882361F1EE2051F120915002822F49
:1019500082958F7090E0029774F080914B02909185
:101960004C0298878F831986BB86AA862C87CE0166
:1019700007960E94D90886E0F801ABE4B2E0019036
:101980000D928A95E1F70E94710B0E94630B0AC0C9
:101990005E1711F1C8010E94440981112CC0C801D1
:1019A0000E94D908FF24F394D1C0282F207F81F70B
:1019B0007A2DB98AA88A6E2D89890E944C098BE4F8
:1019C00092E00E94D90886E0D6011D928A95E9F737
:1019D0000E94630BF12CBAC04913DCCFE110DACFBF
:1019E000F8018583C8010E94D90886E0D6011D92BE
:1019F0008A95E9F7ABC0EE2091F220915002822F38
:101A000082958F7090E002970CF4B5CF80914B02D5
:101A100090914C029A8389831B82BD82AC822E8373
:101A2000CE010196A6CF6217730708F044C0FE2CC2
:101A3000EE2009F4B4CF5E1330C049132EC02091BC
:101A4000500220FD21C0822F82958F70482F50E0D8
:101A500041155105C9F0F80125834F30510541F07A
:101A60008F5F982F9295907F822F8F70892B85831F
:101A7000C8010E94D90886E0F801ABE4B2E0019009
:101A80000D928A95E1F73CC086E0F801ABE4B2E044
:101A900001900D928A95E1F759C0C8010E9444094E
:101AA000811169CF80915002816080935002C801FA
:101AB0000E94D9084BC07A2DB98AA88A6E2D8989CF
:101AC0000E944C0986E0D6011D928A95E9F718C05C
:101AD000EE2009F464CFC8010E944409F82E88233F
:101AE00009F45DCF86E0F801ABE4B2E001900D921D
:101AF0008A95E1F78BE492E00E944A050E94710BFF
:101B00000E94630B23C04D875E878D859E850E9452
:101B1000140B292F22952F70223028F49F7039F052
:101B2000811105C00BC0243028F49F7049F4805EF9
:101B3000883020F0C8010E94D9089F2CF92C06C0DB
:101B4000D80115969C91907F91F7F8CF8F2D6196D3
:101B50000FB6F894DEBF0FBECDBFDF91CF911F91BE
:101B60000F91FF90EF90DF90CF90BF90AF909F903C
:101B700008951F93CF93DF93CDB7DEB72C970FB6A1
:101B8000F894DEBF0FBECDBF4F83588769877A8731
:101B90008B879C87CE0107960E94E90B8823D1F0A2
:101BA0009F8188852A853B85232B31F08F3F31F437
:101BB00081E09F3F19F403C081E001C080E080FD17
:101BC00047C04F81588569857A858B859C850E94A1
:101BD0005B093EC086E0FE013796DE01119601905A
:101BE0000D928A95E1F7FF81E8856A857B8561150D
:101BF000710531F0EF3F31F481E0FF3F19F403C08C
:101C000081E001C080E080FD23C020911A0230E015
:101C1000C9010196877099274091190250E08417F5
:101C20009507F1F1F983EA837D836C8396E0929FB7
:101C3000D001939FB00D1124A55EBD4FFE013196DA
:101C400001900D929A95E1F780931A020E94420B3F
:101C500016E08091190290911A02891771F1189F6C
:101C6000C0011124855E9D4F0E94E90B882329F154
:101C7000E09119021E9FF0011124E55EFD4F4081A5
:101C8000518162817381848195810E945B09809179
:101C9000190290E001968770992780931902D9CF95
:101CA0000E94250910921A0210921902EBE4F2E048
:101CB00086E0DF011D928A95E9F72C960FB6F8941D
:101CC000DEBF0FBECDBFDF91CF911F9108958091F0
:101CD000710285958595859508958091710287702B
:101CE000089590917102977081E009F480E0089561
:101CF00080919402089590919402892B809394028C
:101D00000895809590919402892380939402089578
:101D100010929402089590919302892B80939302DC
:101D2000089580959091930289238093930208955A
:101D300010929302089580917202089508950C9470
:101D40009E0E0C949F0E90911B0392FD08C09091E3
:101D50007202981721F0809372020C94A10E0895DC
:101D600080917202882329F01092720280E00C9414
:101D7000A10E0895CF93DF93E0910201F09103014A
:101D8000809194028083E0910201F091030190819F
:101D900080919302892B808380917202882381F045
:101DA000E0910201F09103019081892B8083809161
:101DB0000201909103010E942E2881110E94B00E11
:101DC000C0910201D091030140E250E061E572E070
:101DD000CE010E94E534892B69F080E2FE01A1E585
:101DE000B2E001900D928A95E1F7CE01DF91CF919B
:101DF0000C94DA27DF91CF9108950C949E0E909168
:101E00001B0392FD10C098E0899F90011124262B9E
:101E1000209371020E94DD0980917102859585955C
:101E200085950C94FD0E0C94DD091092710280E0F2
:101E30000C94FD0E20917102809582238093710293
:101E4000982F977099F430E0482F082E000C550B0E
:101E50002417350759F090911B0392FD07C0859513
:101E6000859585950E94FE090C94150F0895909113
:101E70001B0392FB222720F9281769F080FB92F9B7
:101E800090931B0380911A0390911B030E94850F6E
:101E900082E00C941A0F089580911B0382FB88271F
:101EA00080F991E089270C94370F81E00C94370F6B
:101EB00080E00C94370F6FEF7FEF80E090E00C94A0
:101EC0002D3580E090E00E94093521E0893E9E4F4B
:101ED00009F020E0822F089582E090E00C94FB341A
:101EE00083E090E00C94FB34CF9384E090E00E9478
:101EF000FB34C82F82E290E00E94FB342C2F30E0AC
:101F0000A901582BCA01CF910895CF93C92F682FEB
:101F100084E090E00E940F356C2F82E290E0CF9138
:101F20000C940F35AB01BC018FE090E00C9421358F
:101F3000AB01BC0183E190E00C94213560E070E0DE
:101F4000CB010C94980F60E070E0CB010E94920FDF
:101F50000C949E0F69EE7EEF80E090E00E942D359C
:101F600060E082E090E00E940F3560E083E090E066
:101F70000E940F351092150210921602109217024D
:101F80001092180260E084E090E00E940F3560E05B
:101F900082E290E00E940F3560E085E090E00E94D0
:101FA0000F3560E086E090E00E940F356FEF87E02C
:101FB00090E00E940F3540E050E0BA0188E090E0E8
:101FC0000E94213560E08DE090E00E940F3540E0F6
:101FD00050E0BA0188E190E00E94213560E087E19D
:101FE00090E00E940F3540E050E0BA018CE190E0B3
:101FF0000E94213560E070E080E290E00E942D3583
:1020000040E050E0BA0188E190E00E9421350C9454
:10201000A30F0C94AA0F682F8EE090E00C940F355C
:102020000E9493296093A1027093A2028093A3025D
:102030009093A40260939D0270939E0280939F02EE
:102040009093A002089585B7806885BF85B78068A2
:1020500085BF08950C943C1508950C942C100C9495
:102060002C100C942F100C942C100C9433100C94F6
:102070002C100E94231088E393E10E94BD270E9448
:1020800037100C9435100E942D100C942C100E94C7
:1020900052130C94E4040E947E290E94EE120E94C6
:1020A00056150E948D140E9447100E9437230E94EB
:1020B0002D210E946A150C9431108F929F92AF923D
:1020C000BF92CF92DF92EF92FF920F931F93CF9325
:1020D000DF93CDB7DEB72A970FB6F894DEBF0FBEF9
:1020E000CDBF0E94B114982E81110E94101085E975
:1020F000A82E82E0B82E00E010E0802E802F0E94F3
:102100007613D82EF501C1905F01C826B1F40F5F98
:102110001F4F0830110589F78FEF89838A831B824F
:102120000E9487298160782F9D838C8349815A8101
:102130006B818D810E9400052FC08091A50281FDD9
:102140000E947C13E12CFF24F3948C2D8F21F1F05D
:102150000E942A10882399F0EE828F82DF2081E08E
:1021600009F480E088870E9487298160782F9A8708
:1021700089874E815F8168858A850E940005F80104
:10218000EB56FD4F8081F826F08206C0E394FF0CE9
:10219000F7E0EF12DACFBBCF81E0911001C080E011
:1021A0002A960FB6F894DEBF0FBECDBFDF91CF9158
:1021B0001F910F91FF90EF90DF90CF90BF90AF9065
:1021C0009F908F9008950E945D100E943C150E9480
:1021D00065210E94AE190C94F504CF93DF930E9401
:1021E0001712EC01811521E5920708F045C0811511
:1021F00030E5930708F094C0883E910528F5803EAD
:10220000910508F0F8C0883A910570F4853A910577
:1022100008F07CC08130910509F475C008F4E8C06D
:10222000049708F0E8C0E4C08F3B910508F0E0C0D7
:10223000C85AD0E0CC0FDD1FCA57DE4F0990D881B5
:10224000C02DCE019464D8C0811540E2940758F4A3
:10225000811551E0950708F0CEC08D3E910508F438
:10226000C7C09065C9C0C11580E4D80708F4C0C0D4
:10227000DF70CE01906AC0C0811525E59207A8F4F1
:10228000811534E5930708F095C0811543E594075F
:1022900008F07BC0811552E5950708F061C0D82F82
:1022A000CC27CE01816F906AA7C0C11589E5D807F8
:1022B000A0F4C11528E5D20708F082C0C11536E5A3
:1022C000D30708F095C08C2F0E94AB128F7190E05D
:1022D000D82FCC27CE0190628FC0C1154AE5D40714
:1022E00008F474C0CE0190568115904208F080C069
:1022F0008D2F8F710E94AB12DD27D0628F71AE01DE
:10230000582BCA0179C081E090E076C0C55AD0E070
:10231000CC54DE4F8881C82FD0E0CE0190646CC0D1
:1023200074E0969587957A95E1F7282F23703C2FD6
:10233000337081E090E002C0880F991F3A95E2F770
:102340009C68AC01522B9A019C2F9F709695969594
:1023500050E2959FE0011124C9018C2B9D2B4CC0AC
:102360008370992721E030E002C0220F331F8A9545
:10237000E2F79C2F9695969580E2989FE0011124B4
:10238000C22BD32BCE019C6837C08370992721E0E4
:1023900030E002C0220F331F8A95E2F79C2F9695FA
:1023A000969540E2949FE0011124C22BD32BCE01DD
:1023B0009A6822C0D82FCC27CE01846F906A1CC0A7
:1023C000DC2FCC27CE01806F906A16C08C2F8F70C7
:1023D0000E94AB1294E0D695C7959A95E1F7CF701D
:1023E000D0E0DC2FCC27D0699E01282BC90104C086
:1023F00080E090E001C0CE01DF91CF91089528E305
:10240000829FC0011124FC0127E0729FE00DF11DA5
:102410001124E60FF11DEE0FFF1FEE5CFE4F8591BC
:10242000949108950E94FF110E94ED100895823842
:10243000910569F1B0F48133910509F46DC048F458
:102440008932910509F463C08A32910509F469C0A3
:1024500008958533910509F455C089339105B9F084
:102460000895833E910569F138F4803E9105B1F0FD
:10247000823E910509F10895863E9105A9F1873EB6
:102480009105B9F1843E910509F064C023C0209103
:102490001A0320FD4FC021FD4DC0089580911A03FD
:1024A00080FD44C080911B0380FF44C080911A03CB
:1024B00084FD42C083EE4DC080911A0382FF38C074
:1024C000F5CF80911A0382FD33C080911B0380FDFC
:1024D00031C0ECCF80911B0381FF32C080911A0381
:1024E00084FD2AC087EE35C080911A0383FF26C081
:1024F000F5CF80911A0383FD21C080911B0381FDDC
:102500001FC0ECCF80911A0385FD1CC01DC08091B7
:102510001A0385FD19C016C080911A0386FD16C0E6
:1025200017C080911A0386FD13C010C089E311C043
:1025300082EE0FC080EE0DC080E00BC086EE09C0B9
:1025400084EE07C089E205C085E303C08AE201C0CA
:1025500081E390E0089590911A0392FF0DC0282F17
:102560002871283019F4877F846006C0282F2471D1
:10257000243011F48B7F886093FF0DC0282F2871C1
:10258000283119F4877E846106C0282F24712431F4
:1025900011F48B7E886120911B0320FF0DC0382F22
:1025A0003871383019F4877F816006C0382F317157
:1025B000313011F48E7F886021FF0DC0282F2871E3
:1025C000283119F4877E816106C0282F21712131BD
:1025D00011F48E7E886194FD877E08951092160313
:1025E0001092170310921803109219030895CF92B6
:1025F000DF92EF92FF926B017C010E943C158111EA
:102600000EC00E949329C61AD70AE80AF90AC09296
:102610001603D0921703E0921803F0921903FF906B
:10262000EF90DF90CF9008950F931F930E943C1579
:10263000882321F01F910F910C9493290E949329D4
:10264000009116031091170320911803309119037C
:10265000600F711F821F931F1F910F9108950E9499
:102660003C1581110C9487290E941413CB01089505
:1026700080E008950C945B0F0E94B1148FE39CE9F5
:102680000197F1F700C000000E94B11480E00E94A1
:10269000761380FF04C00E943A130C94F029089529
:1026A0000C943C130E94610F811102C00E9409101A
:1026B0000E946C0F8093A5020E94740F90931B03DD
:1026C00080931A030E9450130E94700F682F70E0CD
:1026D00080E090E00E947D096091110270911202E9
:1026E00080911302909114020C94B509E82FF0E048
:1026F000EB5DFC4F80810895089580EA8A95F1F79B
:10270000089500C008950C947D1308950C948513CA
:102710000C9486130C9485130C948A130C948513D3
:102720000F931F93CF93DF9300D000D0CDB7DEB7C8
:102730000E943C1560912D038823E9F119821A82C9
:102740001B821C82862F90E08E010F5F1F4FB80105
:102750008B5D9C4F0E947815882389F080911C0323
:1027600090E044E050E0B8018B5D9C4F0E94E5345E
:1027700021E02093A602892B69F410E019C0809112
:10278000A6028823D1F384E0F80111928A95E9F733
:102790001092A602E0911C03F0E0EB5DFC4F8981F2
:1027A0009A81AB81BC8180839183A283B38311E042
:1027B0000E9490030DC070E06B5D7C4F80911C0304
:1027C00090E08B5D9C4F0E9458160E948E1310E083
:1027D000812F0F900F900F900F90DF91CF911F914D
:1027E0000F910895F894E82FE295EF70F0E031A191
:1027F000282F2F7081E090E001C0880F2A95EAF71A
:10280000982F9095932391A392A1892B82A37894DA
:1028100008950F931F93CF93DF93CEEBD1E089916F
:102820008F3F11F00E94F21381E0C23CD807B9F744
:10283000C7EBD1E00EEB11E089918F3F11F00E94C0
:10284000F2130C171D07C1F7DF91CF911F910F9164
:102850000895CF92DF92EF92FF920F931F93CF9341
:10286000DF938C01C62FD0E0CE0182549E4F7C01B5
:10287000FC0190819F3F09F447C0D62EF894E92FC0
:10288000E295EF70F0E081A19F7021E030E001C09F
:10289000220F9A95EAF7822B81A382A12095282303
:1028A00022A378940E948113E7EBF1E04EEB51E014
:1028B00031E0C12C21912F3F89F0A22FA295AF705A
:1028C000B0E090968C9190E02F7002C0959587951E
:1028D0002A95E2F780FD02C0832F01C080E0C82A5C
:1028E000330F4E175F0731F7F70180818F3F11F0EB
:1028F0000E94F21361E0C11001C060E08D2D0E94C2
:102900008313C00FD11FC882DF91CF911F910F9108
:10291000FF90EF90DF90CF90089580910401809117
:102920000401811102C094E001C090E090932D0356
:1029300084E0891B80931C030E94091488E0E5E26F
:10294000F3E0DF01982F1D929A95E9F7EDE1F3E0AE
:10295000DF011D928A95E9F784E00E9405150C9429
:102960008E03EF92FF920F931F93CF93DF93CDB718
:10297000DEB728970FB6F894DEBF0FBECDBF8E012D
:102980000F5F1F4F88E0F80111928A95E9F7F12C4B
:102990006F2DC8010E942914F394F4E0FF12F8CFC0
:1029A00048E050E0B8018DE193E00E94E5347C01FD
:1029B00021E0892B09F420E0E114F10441F088E0E2
:1029C000F801ADE1B3E001900D928A95E1F76091D5
:1029D0002D0370E06B5D7C4F44E08DE193E00E943D
:1029E0000615EF2819F40E94901302C081E090E0D0
:1029F00028960FB6F894DEBF0FBECDBFDF91CF9102
:102A00001F910F91FF90EF9008950895FF920F93FB
:102A10001F93CF93DF938C01F62ED72FC42F222341
:102A200049F081E08093A9020E9487299093A8022F
:102A30008093A7028091A9028823C1F08091A70208
:102A40009091A8020E949F29059780F0EF2DFD2FFD
:102A5000D8014C2F50E0CD01801B910B84179507B6
:102A60001CF48D918193F7CF1092A902DF91CF9141
:102A70001F910F91FF9008958091AC0281110DC0BC
:102A80000E94E730811102C082E001C081E08093A2
:102A9000AC02823011F40E94E23081E09091AC02ED
:102AA000913009F080E008950C943C150E94541573
:102AB000809304018091040165E0882311F080E097
:102AC00001C085E00E94641B0E943C1581110C949A
:102AD000B01508950E943C15811102C00C94B215E6
:102AE000089581E09091AD029A3008F080E0089559
:102AF0000F931F93CF93DF93EC018B018091AD0275
:102B00008A3038F4B801CE010E94561681111DC0DA
:102B10000AC08091AA029091AB020E949F29843F33
:102B2000914080F715C08091AD028F3F19F08F5F03
:102B30008093AD028091AD028A3060F00E948729B7
:102B40009093AB028093AA0203C01092AD0202C020
:102B500080E001C081E0DF91CF911F910F91089536
:102B60000C948D2582E30C9407270F931F9398E014
:102B70008902F0011124EB5FFE4F26813781232B60
:102B800091F08093510360910601709107012091AB
:102B9000050130E0AB014F5A5C4F04E610E082E3E0
:102BA0000E948E2602C080E090E01F910F91089550
:102BB0005F926F927F928F929F92AF92BF92CF92CD
:102BC000DF92EF92FF920F931F93CF93DF93582ED4
:102BD00069015801C82F880FDD0B4115510531F4EB
:102BE000852D0E94B51597FF28C025C0CE0123E092
:102BF000880F991F2A95E1F7FC01EB5FFE4FE080FB
:102C0000F12C4E155F0508F47A01FC01EB5FFE4FD5
:102C100081809280C4018F5A9C4F3C01A7010E9481
:102C2000F23404E610E09701A301682D82E30E94CC
:102C30008E2697FFD5CF80E029C0A114B10429F1D9
:102C400083E0CC0FDD1F8A95E1F7FE01EB5FFE4FBD
:102C5000E380F12CAE14BF0408F47501CB5FDE4FA6
:102C60006C817D81AB014F5A5C4F04E610E0970107
:102C700082E30E94BB2697FDDECF6C817D816F5A77
:102C80007C4FA701C6010E94F23481E0DF91CF9111
:102C90001F910F91FF90EF90DF90CF90BF90AF907A
:102CA0009F908F907F906F905F9008950C94C417C1
:102CB0000C94E8170F931F93CF93DF9300D000D0AD
:102CC000CDB7DEB76091BA027091BB028091BC02B1
:102CD0009091BD020E94AE2964367105810591056F
:102CE00028F10E941413DC01CB010296A11DB11D35
:102CF00089839A83AB83BC8300E010E020E030E05E
:102D000044E050E0BE016F5F7F4F83E00E94D81522
:102D1000182F882361F00E9493296093BA02709360
:102D2000BB028093BC029093BD0201C011E0812FD1
:102D30000F900F900F900F90DF91CF911F910F91F7
:102D40000895AF92BF92CF92DF92EF92FF920F93CE
:102D50001F93CF93DF937C015B016A010E94711581
:102D6000811103C001E010E002C00AE010E0C1E000
:102D7000D0E0F894B501C701F60109957894811166
:102D800015C021960C171D0794F0CC9F9001CD9F84
:102D9000300D300D112480E090E045E34A95F1F7C5
:102DA0000000019682179307C1F7E3CF81E0DF911E
:102DB000CF911F910F91FF90EF90DF90CF90BF9038
:102DC000AF9008950F931F93CF93DF93CDB7DEB7E6
:102DD00028970FB6F894DEBF0FBECDBFCE01019687
:102DE0000E94FE1F18856091BE027091BF02809103
:102DF000C0029091C1020E94AE296436710581051E
:102E0000910510F41123D9F000E010E020E030E04B
:102E100048E050E0BE016F5F7F4F84E00E94D8150C
:102E2000882359F00E9493296093BE027093BF02D9
:102E30008093C0029093C10202C080E003C00E9450
:102E4000FB1F81E028960FB6F894DEBF0FBECDBF02
:102E5000DF91CF911F910F910895AF92BF92CF92C2
:102E6000DF92EF92FF920F931F93CF93DF9300D0E7
:102E700000D01F92CDB7DEB75B01E090C201F090A9
:102E8000C30101E010E09E012B5F3F4F40E050E0A6
:102E900060E070E081E00E94D815182F882309F4C3
:102EA0003EC0670182E0C80ED11C6091B6027091ED
:102EB000B7028091B8029091B9020E94AE2964369F
:102EC00071058105910518F104E010E09E012F5F66
:102ED0003F4F40E050E060E070E082E00E94D81593
:102EE000182F64E070E0C6010E94382391E02D8124
:102EF000281390E0192351F10E9493296093B602A0
:102F00007093B7028093B8029093B90211C064E045
:102F100070E0C6010E9438239D818913D5CFF70147
:102F200082819381A481B58189839A83AB83BC8399
:102F3000112361F089819A81AB81BC818093B202B7
:102F40009093B302A093B402B093B5028091B20201
:102F50009091B302A091B402B091B502F5018083C3
:102F60009183A283B383812F0F900F900F900F90C6
:102F70000F90DF91CF911F910F91FF90EF90DF9015
:102F8000CF90BF90AF9008950F931F93CF93DF938F
:102F9000EC018B014DE257E10E94A116882391F0CC
:102FA0004AE556E1B801CE010E94A116882351F0EE
:102FB00042EE56E1B801CE01DF91CF911F910F9102
:102FC0000C94A11680E0DF91CF911F910F9108958D
:102FD0000F931F93CF93DF93F894C091C201D091C8
:102FE000C301CE01029624E0FB01DC0101900D92A9
:102FF0002A95E1F764E070E00E9438238983789491
:10300000F8946E817F81888599850091AE02109138
:10301000AF022091B0023091B102601771078207B0
:10302000930751F06093AE027093AF028093B002A9
:103030009093B1020E94F7127894F89489898823BA
:1030400031F060E0CE010A960E94F820198A789447
:10305000DF91CF911F910F9108950E94A82B0E949C
:103060004B100C94B42B0E94B82B0E94E3100C94CC
:10307000D22B0E9425290E948F2B0E9439100E947A
:103080002D180E9433180E944310FBCF8091C80274
:1030900080FF06C06091320170E0660F771F26C086
:1030A00081FF04C06091320184E005C082FF07C047
:1030B0006091320188E0689FB001112417C090919F
:1030C000C7029923D1F060913101961788F72091BA
:1030D000320188E0289F90011124929FA001939FC4
:1030E000500D112470E0CA010E945F3460387105F0
:1030F00040F46115710519F406C068E070E0862F90
:1031000008958FE7089581E008958091C80280FFB7
:1031100008C060912E0170E075956795759567956B
:1031200021C081FF06C060912E0170E07595679502
:1031300019C082FF04C060912E0170E010C0909110
:10314000C602992399F060912D019617A0F78091FE
:103150002E01899FC001112470E00E945F34603805
:10316000710540F46115710519F406C061E070E065
:10317000862F08958FE7089581E008958D3E21F40C
:103180000E944618819504C08E3E29F40E9446187C
:103190008093CC0208958F3E21F40E9446188195B9
:1031A00004C0803F29F40E9446188093CB02089502
:1031B000893F19F40E94851805C08A3F31F40E94A6
:1031C000851881958093CD0208958B3F21F40E944C
:1031D0008518819504C08C3F29F40E94851880933E
:1031E000CE0208959FE0980F983078F421E030E007
:1031F000A90102C0440F551F9A95E2F7CA019091A8
:10320000CA02892B8093CA0208958D3F21F48091D0
:10321000C80281600BC08E3F21F48091C802826099
:1032200005C08F3F29F48091C80284608093C80252
:1032300008958D3E39F49091CC0297FF35C01092DD
:10324000CC0259C08E3E29F49091CC021916BCF3E1
:103250002BC09091CB028F3E29F497FF25C010928E
:10326000CB0249C0803F19F41916CCF31DC09091D0
:10327000CD02893F29F41916BCF41092CD023BC04F
:103280008A3F19F497FF10C0F8CF8B3F39F4909123
:10329000CE0297FF09C01092CE022DC08C3F21F4C0
:1032A0009091CE021916BCF39FE0980F983080F4ED
:1032B00021E030E0A90102C0440F551F9A95E2F7C2
:1032C000CA0180959091CA0289238093CA0213C0D3
:1032D0008D3F21F48091C8028E7F0BC08E3F21F478
:1032E0008091C8028D7F05C08F3F29F48091C8026C
:1032F0008B7F8093C8028091CB02811106C08091A0
:10330000CC02811102C01092C7028091CD028111BE
:1033100006C08091CE02811102C01092C6020895AB
:103320000E9487292091CB02211104C02091CC0258
:10333000222321F09093C5028093C4022091CD02F4
:10334000211104C02091CE02222321F09093C302C8
:103350008093C20289EC92E00C94F427EF92FF92E2
:103360000F931F93CF93DF9300D000D000D0CDB741
:10337000DEB786E0E9ECF2E0DE01119601900D92F5
:103380008A95E1F7E090CB02F090CC020091CD025B
:103390001091CE021092CB021092CC021092CD026C
:1033A0001092CE02E11003C0FF2009F45DC08091AD
:1033B000C4029091C5020E949F29AC019091C7025E
:1033C000992339F02091330130E02417350758F064
:1033D0004BC0209134018AE0289F900111242417CA
:1033E000350718F041C09F3F19F09F5F9093C702C7
:1033F000EE2061F00E9446181E1414F09FEF01C0E9
:1034000091E0989F902D11249093CB02FF2061F0C2
:103410000E9446181F1414F09FEF01C091E0989F7E
:10342000902D11249093CC023091CB023323E1F004
:103430002091CC022223C1F045EB3403C0011124BA
:10344000992319F09093CB0203C081E08093CB02C3
:1034500035EB2303C0011124992319F09093CC027A
:1034600003C081E08093CC02011103C0112309F451
:103470005DC08091C2029091C3020E949F29AC015D
:103480009091C602992339F020912F0130E0241742
:10349000350758F04BC0209130018AE0289F9001F9
:1034A00011242417350718F041C09F3F19F09F5F82
:1034B0009093C602002361F00E948518101614F044
:1034C0009FEF01C091E0989F902D11249093CD0221
:1034D000112361F00E948518111614F09FEF01C0AE
:1034E00091E0989F902D11249093CE023091CD02BF
:1034F0003323E1F02091CE022223C1F045EB3403C7
:10350000C0011124992319F09093CD0203C081E0EA
:103510008093CD0235EB2303C0011124992319F0C8
:103520009093CE0203C081E08093CE028091CB02C3
:1035300081110BC08091CC02811107C08091CD0216
:10354000811103C08091CE0281110E949019EB82FB
:10355000FC820D831E8386E0FE013196A9ECB2E069
:1035600001900D928A95E1F726960FB6F894DEBF8A
:103570000FBECDBFDF91CF911F910F91FF90EF90C4
:103580000895E9ECF2E086E0DF011D928A95E9F703
:103590001092C7021092C6021092C8020895EF92CC
:1035A000FF920F931F93CF93DF938B01682F11111D
:1035B0000AC0442329F0E82FF0E0E754FC4F64915F
:1035C000762F862F75C0212F30E0E82FF0E04423BE
:1035D00021F0E754FC4FE491F0E046E0049FC00185
:1035E0001124CFEFD0E0BE010E944B344BEA4603DA
:1035F000C001479F900D1124800F911D800F911DD8
:10360000982F990F890FAE01421B530B4E9FD0018B
:103610004F9FB00D5E9FB00D11249B2F189FA001EE
:103620001124452F55278E01041B150B0E9FA00159
:103630000F9F500D1E9F500D11247E01E81AF108B6
:10364000E29E8001E39E100DF29E100D1124212FA9
:103650003327C21BD30BCE9F9001CF9F300DDE9F2F
:10366000300D112462307105A9F048F4611571051F
:1036700069F061307105C9F48B2F752F0DC064306E
:10368000710581F058F06630710579F47E2F8B2F2B
:10369000932F0DC0832F7B2F9E2F09C08E2F7B2F42
:1036A000952F05C08E2F732F02C07E2F852F692F77
:1036B000DF91CF911F910F91FF90EF90089541E01E
:1036C0000E94CF1A08950895E8E3F1E080836183B2
:1036D00008950E945F1B0895CF93DF93762FE90131
:1036E000682F842F0E94691B798368838A83DF9106
:1036F000CF91089580912E03282F269530E0211533
:10370000310519F48170826005C02532310524F03D
:103710008170886480932E03089588E090E00C9473
:103720000335CF92DF92EF92FF926B017C010E94F2
:103730007A1BB701A60188E090E0FF90EF90DF9040
:10374000CF900C942135EEE2F3E083E08083118288
:103750008FEF828383831482AEEDB2E012968C9158
:103760001297836012968C9360817181828193811C
:103770000C94911B80912E0380FF02C086950895C2
:1037800080E0089590913203933018F49F5F9093F6
:103790003203882351F060912E0370912F038091A2
:1037A0003003909131030C94911B089581E00C94A7
:1037B000C21B90913203992319F0915090933203D8
:1037C000882351F060912E0370912F038091300374
:1037D000909131030C94911B089581E00C94D91BB6
:1037E00070E00C940C236091390180912E0380FFCE
:1037F0000AC08091380123E0829FC00111248D5CB2
:103800009C4F0C94F01B80913A0190913B018917D9
:1038100080F7E82FF0E09F01220F331FE20FF31F24
:10382000ED5CFC4F1182108212828F5FF0CF90917D
:103830002E0390FF16C090913A0120913B01921700
:1038400070F4E92FF0E0DF01AA0FBB1FEA0FFB1FA6
:10385000ED5CFC4F8183608342839F5FF0CF0C94CB
:10386000F31B0895CF93DF9300D01F92CDB7DEB73F
:1038700090912E0390FF0AC09E012F5F3F4F0E9440
:103880006C1B4B8169818A810E94171C0F900F90DD
:103890000F90DF91CF910895CF93DF93EC016C816E
:1038A00070E080E090E00E943E3220E030E04FE7A0
:1038B00053E40E9461312BED3FE049E450E40E9463
:1038C00067330E94D4330E94DB312BE43AE34EE2AB
:1038D0005FE30E94F43020EF3BEF48ED52E40E949A
:1038E00067330E940D32462FEEE2F3E06281818160
:1038F0000E94321C8C818F5F8C83DF91CF91089561
:10390000CF93DF93EC01EEE2F3E0438162818C819F
:103910000E94321C8C818F5F8C83DF91CF91089540
:103920000F931F93CF93DF9300D01F92CDB7DEB7D5
:103930008C018091CF0281110AC09E012F5F3F4F01
:103940004FEF6FEF0E946C1B8A818093CF02F801CA
:103950008481813051F028F0823061F44091CF02AF
:103960000AC08091CF0240E007C06091CF0240E0E2
:1039700080E003C040E080E060E00E94171CF80196
:10398000848190E0019663E070E00E945F3484835C
:103990000F900F900F90DF91CF911F910F9108958D
:1039A000AF92BF92CF92DF92EF92FF920F931F934D
:1039B000CF93DF9300D01F92CDB7DEB7182FF62E2E
:1039C000042FE22E90912E0390FF7EC0E92FE69502
:1039D000AE2FB0E0AC53BE4F8C918093DE029E7F41
:1039E000923061F49E012F5F3F4F812F0E946C1B2C
:1039F0004B8169818A810E94171C43C0823019F46F
:103A0000009131033EC0863019F410912F0339C064
:103A10008930D9F38931A9F5E9518E2F8170D82EDB
:103A2000E695F0E0EC54FC4FA590B490C12CBB247B
:103A300060913C01C61618F52C2D30E0A29EC00105
:103A4000A39E900DB29E900D112470E00E944B3405
:103A5000812FD11002C0860F01C0861B90913A01C0
:103A6000290F311DA901440F551F240F351F2D5C4F
:103A70003C4F402F6F2D0E946C1BC394D9CF0E94E6
:103A8000F31B80912F03181308C080913003F812A4
:103A900004C080913103081729F08091E002826010
:103AA0008093E00210932F03F092300300933103D0
:103AB000EE2051F060912E0370912F03809130031E
:103AC000909131030E94911B0F900F900F90DF9106
:103AD000CF911F910F91FF90EF90DF90CF90BF900B
:103AE000AF900895EEE2F3E09181282F4381628147
:103AF00088E0890F0C94D01C81E00C94721DEEE2DA
:103B0000F3E09181282F4381628188EF890F0C9423
:103B1000D01C81E00C947F1DEEE2F3E0628128E08E
:103B2000620F08F46FEF282F438181810C94D01C21
:103B300081E00C948C1DEEE2F3E0628128E0621BD0
:103B400008F460E0282F438181810C94D01C81E02F
:103B50000C949B1DEEE2F3E0438128E0420F08F451
:103B60004FEF282F628181810C94D01C81E00C944E
:103B7000AA1DEEE2F3E0438128E0421B08F440E096
:103B8000282F628181810C94D01C81E00C94B91D96
:103B900020E00C94D01CFF920F931F93CF93DF93E0
:103BA000EC01F12C0FEF10E060913C01F616F0F4FF
:103BB00080913A012F2D30E0280F311DC901880F67
:103BC000991F280F391F2D5C3C4F70E0C8010E94DF
:103BD0005F34962F8C814091310360913003F99EC0
:103BE000800D11240E946C1BF394DECF0E94F31B06
:103BF0009A818C8190FF02C08F5F01C081508C83BD
:103C0000DF91CF911F910F91FF9008958F929F9216
:103C1000AF92BF92CF92DF92EF92FF920F931F93DA
:103C2000CF93DF93EC018A8180FF03C0BB24BA9459
:103C300002C0BB24B3948C8181110DC081E0B81205
:103C400006C080913C0181508093D10202C0109245
:103C5000D10281E08C83A12C4AE0942E80913C011A
:103C6000A81608F044C080913A01CA2CD12C8601D4
:103C7000080F111DC801880F991F080F191F0D5C2F
:103C80001C4FF80111821082128234E0E32EF12CD5
:103C9000812C8091D102880D8B302CF0692D0E94EF
:103CA0003D34892F05C087FF03C090913C01890FE7
:103CB000082E000C990BC816D90691F48091310397
:103CC0008E9DA0018F9D500D1124559547955595BA
:103CD000479598016091300380912F030E946C1BDF
:103CE0008B0CF1E0EF1AF108A1F6A394B7CF0E9474
:103CF000F31B8091D10291E0B9120EC0811107C06F
:103D000080913C0181508093D1021C820FC0815070
:103D10008093D102BC820AC090E0019660913C0180
:103D200070E00E945F348093D1028C83DF91CF9149
:103D30001F910F91FF90EF90DF90CF90BF90AF90C9
:103D40009F908F9008951F93CF93DF93EC018C8108
:103D5000811109C081E08C831092D00292E090938F
:103D600037018093360180913A0190913B01891788
:103D700070F4E82FF0E09F01220F331FE20FF31FD2
:103D8000ED5CFC4F1182108212828F5FF0CF10E049
:103D900060913C011617C0F5E12FF0E070E0CF0113
:103DA0000E945F3420913A01820F2091D002022EAE
:103DB000000C330B90E0E217F307CCF020913701B1
:103DC000022E000C330B2E173F078CF09C01220FA4
:103DD000331F820F931F9C012D5C3C4F4091310398
:103DE0006091300380912F030E946C1B0BC0FC017B
:103DF000EE0FFF1F8E0F9F1FFC01ED5CFC4F118229
:103E0000108212821F5FC4CF0E94F31B8091360183
:103E10002091D002280F2093D00290913701980F63
:103E20009093370119165CF4022E000C330B40916D
:103E30003C0150E0415051092417350734F0819579
:103E400080933601813009F41C82DF91CF911F915C
:103E500008958F929F92AF92BF92CF92DF92EF928E
:103E6000FF920F931F93CF93DF938C01FC0144814A
:103E7000C42FD0E09E01DE010E94A3349B01AC015F
:103E80000E94B9346B017C01E0E2F0E0EC1BFD0B19
:103E9000A5E5B0E09B01AC010E94B9344B015C0187
:103EA0009F01DF010E949B349B01AC010E94C4343E
:103EB0009B01AC012C0D3D1D4E1D5F1DC501B401C4
:103EC0000E947334C22FD22F2A3228F4F3E02F9F9E
:103ED000900111240DC025E530E02C1B3109C901EA
:103EE000880F991F280F391F37FF02C02F5F3F4FE0
:103EF00035952795C22FC095F12C85E5E82EED1A52
:103F000080913C01F816C8F4F1FC02C08E2D01C06E
:103F10008D2F90913A012F2D30E0290F311DA901ED
:103F2000440F551F240F351F2D5C3C4F4C2F6091C3
:103F300030030E946C1BF394E3CF0E94F31BF80143
:103F40008481811102C091E003C0803219F49FEF97
:103F50009093350190913501890FF8018483DF91A9
:103F6000CF911F910F91FF90EF90DF90CF90BF9076
:103F7000AF909F908F9008950F931F93CF93DF93EF
:103F8000EC0100E010E080913C01282F30E00217A6
:103F9000130724F590913A019801290F311DA901C9
:103FA000440F551F240F351F2D5C3C4F869590E024
:103FB0004C81081719071CF4442331F002C0411149
:103FC00003C04091310301C040E060913003809113
:103FD0002F030E946C1B0F5F1F4FD5CF0E94F31B56
:103FE0008C8190E00196817099278C83DF91CF912D
:103FF0001F910F9108951092E002089525E0EEE2DE
:10400000F3E0DC0101900D922A95E1F72091DE02A8
:104010003091DF024091E002FC0125833683478323
:10402000089560912E03669570E04BE050E08DE3BB
:1040300091E00E94D834892B19F481E08093DF024B
:104040000E942F139093D6028093D5028091E002B4
:1040500084608093E0020895EEEDF2E011828281A7
:1040600084608283089590912E0390FF3AC09170EE
:10407000811102C0926006C0853210F0986402C0BF
:10408000880F982B90932E038091E002816080939B
:10409000E002662351F060912E0370912F0380910E
:1040A0003003909131030E94911B60912E0366951D
:1040B00070E04BE050E08DE391E00E94D834892B12
:1040C00019F00E942C2002C00E94112081E08093F0
:1040D000D802409131036091300380912F030C94FA
:1040E000C81D0895682F90912E03969581E0890F41
:1040F000853208F081E00C94332081E00C9472202A
:10410000682F90912E0396958FEF890F09F484E222
:104110000C94332081E00C94802061E00C943320D7
:10412000EEE2F3E080818160808386950C948D209F
:1041300060E00C943320EEE2F3E0808181608083C4
:1041400086950C9498201092DC028091DB028111FC
:104150000E949B200C941120EEE2F3E080818E7F80
:10416000808360817181828193810E94911B0E9472
:104170002C20EEEDF2E08281816082832FEF80E7D8
:1041800092E0215080409040E1F700C000000C9484
:10419000F31B80912E0380FD0C94AC200C94902096
:1041A000EEE2F3E080818E7F80830E942C20EEED92
:1041B000F2E08281816082832FEF80E792E02150DC
:1041C00080409040E1F700C000000C94F31B0E9477
:1041D0002C208091DC0281110AC081E08093DC02F6
:1041E00080912E0381708093DB020C94D02008957F
:1041F0001F93CF93DF93EC01162F8F8180FF0FC0A9
:10420000888180FF0AC080912E03816080932E03F5
:10421000888186950E94332002C00E94D0208F8121
:1042200081FF06C0212F4B816A8189810E94D01CA9
:104230008F8182FF08C08E81882319F00E9411208F
:1042400002C00E942C208F8183FF03C081E08093F5
:10425000D802DF91CF911F9108958091DD028111E5
:1042600033C00E94610F811104C00E9409100E9496
:10427000A31B0E948D1B60932E0370932F038093CA
:104280003003909331038091E00283608093E002D9
:104290006E7F61F40E94A31B0E948D1B60932E030E
:1042A00070932F0380933003909331030E947A1B05
:1042B0000E942C2080912E0380FF03C086950E94CF
:1042C000982081E08093DD020895EF92FF920F9392
:1042D0001F93CF93DF938091DF02882309F4ABC053
:1042E0008091DE02E0912E03E695E81BE093D70271
:1042F000823049F4F0E0E055FC4FE491CE2FD0E05D
:104300000CE41CE149C0863049F4F0E0E355FC4F71
:10431000E491CE2FD0E000E81CE13EC0893051F49A
:10432000E695F0E0E655FC4FE491CE2FD0E00BECA3
:104330001DE132C08F3051F4E695F0E0E955FC4FB5
:10434000E491CE2FD0E006E01EE126C0853149F48D
:10435000F0E0EC55FC4FE491CE2FD0E003EA1EE1F3
:104360001BC0883181F0833239F4E2EAF3E0C59171
:10437000D49100E91CE110C0843251F4C4EFD1E0C3
:104380000CEB1FE109C0C8E2D0E009E21FE104C064
:10439000C0EDD7E003E61BE18091D802882361F0ED
:1043A0001092D8020E942F139093D6028093D502C8
:1043B0001092DA021092D9020E942F13E091D502D6
:1043C000F091D6029C012E1B3F0B2F3F3F4798F5E3
:1043D0002091D4022223B1F01092D4022091D20273
:1043E0003091D302821B930B8F3F9F4758F4205D7F
:1043F0003A483093D3022093D2028091E002886041
:104400008093E002E090D902F090DA02EC0FFD1FF9
:10441000F093D602E093D50285ED92E0F80109957C
:104420008091D9029091DA02892B29F4EF2819F0B2
:1044300081E08093D402DF91CF911F910F91FF9083
:10444000EF900895882311F0FA0101C0FB0109944F
:10445000CF93DF93C82FD62F0E94BA1B8C1740F042
:104460000E94BA1B8D1720F4DF91CF910C947D2010
:104470008C2FDF91CF910C948D201F93CF93DF93DE
:10448000FB0112811111C3C0EC010E94780E8272EF
:10449000CD3CFCE5DF0709F49AC0A8F5C73CECE584
:1044A000DE0709F476C0A8F4C43C9CE5D90709F4FA
:1044B0005FC028F4C33CDC4509F457C054C0C53C78
:1044C0009CE5D90709F459C0C63CDC4509F45CC039
:1044D0004AC0CA3CFCE5DF0709F46AC050F4C83C96
:1044E000ECE5DE0709F45AC0C93CDC4509F45BC0C1
:1044F0003AC0CB3C9CE5D90709F45FC0CC3CDC4515
:1045000009F460C030C0C23DFCE5DF0709F46FC0AC
:1045100088F4CF3C9CE5D90709F460C008F45CC07E
:10452000C03DFCE5DF0709F45CC0C13DDC4509F492
:104530005BC019C0C53D9CE5D90709F460C050F4C3
:10454000C33DFCE5DF0709F455C0C43DDC4509F473
:1045500054C009C0C63D9CE5D90709F455C0CE3505
:10456000DD4509F454C011E052C00E94C9204FC07B
:104570004AE850E26DE770E204C04DE750E26AE8B5
:1045800070E20E94222243C049E85DE16CE77DE1D0
:10459000F8CF4CE75DE169E87DE1F3CF47EA5DE103
:1045A00068E97DE1EECF48E95DE167EA7DE1E9CFC9
:1045B00045EC5DE166EB7DE1E4CF46EB5DE165EC6A
:1045C0007DE1DFCF4DEE5BE166ED7BE1DACF46EDDD
:1045D0005BE16DEE7BE1D5CF81E017C065E082E065
:1045E00010C068E086E00DC06EE089E00AC064E1BA
:1045F0008FE007C067E185E104C088E106C062E2A0
:1046000089E10E94282203C083E20E948D20812F2D
:10461000DF91CF911F910895259A25B12F7D35B156
:1046200030624FB7F894FC01CB01880F991F680FD7
:10463000791F6E0F7F1FE617F70789F0819198E0C9
:1046400035B9000000C087FF25B9880F000000C001
:1046500000C000C025B900C09A9591F7ECCF4FBFBC
:104660008FE594E00197F1F700C0000008950895E8
:10467000FC01680F791F8FEF91E3E617F70771F0E0
:104680002191822728E030E087FF03C0880F892727
:1046900001C0880F21503109B9F7EFCF0895CF93AA
:1046A000DF93EC01FB018281882309F43CC1C43013
:1046B000FDE5DF0760F4CB3F9CE5D90788F49E0158
:1046C00022503C452431310508F02EC109C0C236C4
:1046D000EDE5DE0729F0C63AFDE5DF0709F024C164
:1046E0000E94740F90931B0380931A03C1318CE5D1
:1046F000D80709F4C6C008F042C0C930ECE5DE07AF
:1047000009F49BC000F5C5308CE5D80709F485C0D5
:1047100078F4C330ECE5DE0709F478C008F07AC01D
:10472000C230DC4509F0F5C080911A038160EFC00A
:10473000C7309CE5D90709F478C008F07AC08091A9
:104740001A038061E4C0CD30FCE5DF0709F487C0BF
:1047500058F4CB309CE5D90709F479C008F07BC048
:1047600080911A0388606FC0CF30FCE5DF0709F441
:1047700080C008F082C080911A03877FC8C0CE3FF6
:104780009CE5D90709F471C000F5C531FCE5DF07E8
:1047900009F485C068F4C3319CE5D90709F475C0F4
:1047A00008F095C00E94250980911A038F77AFC049
:1047B000CC3FFCE5DF07A9F108F054C0CB3FDC4556
:1047C00009F0A7C080911B0340C0C230EDE5DE07B1
:1047D00009F489C058F4C1158DE5D80709F45AC009
:1047E00008F069C080911B0382602FC0C236EDE5DE
:1047F000DE0709F47CC0C63AFDE5DF0709F481C095
:10480000C330DD4509F085C080E06EC080911A0399
:1048100082607DC080911A0316C080911A0388605F
:1048200076C080911B0382604FC080911A03806222
:104830006EC080911A0380646AC00E94250980912D
:104840001A03806864C0846062C081603DC080914A
:104850001A038E7F5CC080911A038D7F58C08091AF
:104860001A0316C080911B0318C080911B038D7F13
:104870002BC080911A038F7E4AC080911A038F7DCE
:1048800046C080911A038F7B42C080911A03877FB4
:104890008B7F3DC080911B038D7F8E7F15C08091E3
:1048A0001A0382FB222720F991E0922790FB82F9DC
:1048B00090FB83F92CC080911B03982F90959170E9
:1048C0008E7F892B90FB81F980931B0322C00E946D
:1048D000250980911A0387FB222720F991E092276E
:1048E00090FB87F914C081E00E940B1012C08091E8
:1048F0001A0384FB222720F991E0922790FB84F988
:1049000006C080911A03982F909590FB80F98093B0
:104910001A0380911A0390911B030E94850F0E9435
:10492000250980E001C081E0DF91CF910895CF9308
:10493000DF9386319C4541F5EB010E94780E982F5C
:104940008A812091020130910301882379F09A7ABB
:1049500081E009F480E08093E102911102C069E2F4
:1049600001C065E3C9010E94C4280AC08091E10228
:10497000811102C069E201C065E3C9010E94CF282C
:104980000E94BA0E80E001C081E0DF91CF910895CE
:104990000F931F93CF93DF93C42FD22FFC018281FB
:1049A0008823C9F04093E4020E9487299093E30290
:1049B0008093E20280E28C0F883008F057C0C77005
:1049C00081E001C0880FCA95EAF7DF91CF911F916E
:1049D0000F910C9482068091E402481330C08091BC
:1049E000E2029091E3020E949F29883C910538F5EC
:1049F00010E21D0FCD17B9F080E28C0F883040F423
:104A0000C77081E001C0880FCA95EAF70E94890645
:104A1000183028F581E09D2F977001C0880F9A9576
:104A2000EAF70E948206802F0E9479061830F0F47F
:104A3000D77081E001C0880FDA95EAF70AC080E2FA
:104A40008C0F883098F4C77081E001C0880FCA9538
:104A5000EAF7DF91CF911F910F910C948906802F77
:104A6000DF91CF911F910F910C947906DF91CF9137
:104A70001F910F9108950F939C01CB01243F4CE5AA
:104A8000340731F188F4293DFCE53F07D9F02A3D90
:104A90004CE5340779F1283D3C45A9F506E221EEC5
:104AA00041EE68ED7CE52BC0263FFCE53F07E1F0D9
:104AB000A8F0273F3C4539F507E225EE46EE67EFC3
:104AC0007CE51DC007E225EE45EE69ED7CE517C0EB
:104AD00006E221EE40EE64EF7CE511C007E225EE30
:104AE00044EE65EF7CE50BC006E221EE42EE66EF98
:104AF0007CE505C008E221E045EE6AED7CE50E9418
:104B0000C82480E008C0FC018281882319F010923B
:104B1000E40201C081E00F9108951092B90088E489
:104B20008093B80008959F92AF92BF92CF92DF9288
:104B3000EF92FF920F931F93CF93DF93B82EEB0169
:104B40000E9487296C01C431D10558F0CF3F8FEF07
:104B5000D80759F0CE0164E170E00E944B347B012C
:104B600007C0EE24E394F12C03C025E0E22EF12CE3
:104B700084E8A82E94EA992E1092BC009092BC0072
:104B80000E9487298C018091BC0087FD08C00E948B
:104B90008729801B910B8E159F05A8F32AC0809151
:104BA000B900887F883041F08091B900887F8031DA
:104BB00019F00FEF1FEF1FC0B092BB00A092BC0016
:104BC0000E9487298C018091BC0087FD08C00E944B
:104BD0008729801B910B8E159F05A8F30AC0809131
:104BE000B900887F883111F0803419F700E010E0B7
:104BF0000EC00EEF1FEFCF3F8FEFD80709F4BCCFE9
:104C0000C6010E949F298C179D0708F4B5CFC801E3
:104C1000DF91CF911F910F91FF90EF90DF90CF9098
:104C2000BF90AF909F9008950F931F93CF93DF9302
:104C3000EB018093BB0084E88093BC000E9487292D
:104C40008C018091BC0087FD0EC0CF3F8FEFD8074D
:104C5000C1F30E948729801B910B8C179D0788F355
:104C60008EEF9FEF0CC02091B900287F81E090E08B
:104C7000283211F480E090E0919581959109DF91BF
:104C8000CF911F910F9108950F931F93CF93DF93AF
:104C9000EC0184EC8093BC000E9487298C018091F8
:104CA000BC0087FD0EC0CF3F8FEFD807C1F30E9435
:104CB0008729801B910B8C179D0788F38EEF9FEF40
:104CC00003C08091BB0090E0DF91CF911F910F91C5
:104CD00008950F931F93CF93DF93EC0184E88093A3
:104CE000BC000E9487298C018091BC0087FD0EC00A
:104CF000CF3F8FEFD807C1F30E948729801B910B0C
:104D00008C179D0788F38EEF9FEF03C08091BB0047
:104D100090E0DF91CF911F910F910895CF92DF9294
:104D2000EF92FF920F931F93CF93DF93C62F6A01E9
:104D30007901B8010E94932597FD11C0B8018C2F0D
:104D40000E941426E601EC0CFD1CCE15DF0539F09F
:104D500097FD05C0B80189910E941426F6CF24E979
:104D60002093BC00DF91CF911F910F91FF90EF90A6
:104D7000DF90CF900895CF92DF92EF92FF920F9342
:104D80001F93CF93DF93D82EC62E7A01E901B80185
:104D90000E94932597FD2AC0B8018C2D0E941426ED
:104DA00097FD24C0B8018D2D81600E949325670175
:104DB000219796012E193F092C173D0768F497FD9E
:104DC00015C0C8010E94442697FD02C0F6018083E9
:104DD000FFEFCF1ADF0AEDCF97FD08C0C8010E9490
:104DE000692697FD03C0CE0DDF1D888324E920933B
:104DF000BC001816190614F480E090E0DF91CF9102
:104E00001F910F91FF90EF90DF90CF9008958093C6
:104E1000BA0085EC8093BC0008951F920F920FB6E4
:104E20000F9211242F933F934F935F936F937F9330
:104E30008F939F93AF93BF93CF93DF93EF93FF93A2
:104E40008091B900887F803899F058F4882309F45C
:104E500074C0803609F073C01092E5021092E70228
:104E60006EC0883A09F45BC0883B09F458C067C03B
:104E70008091E50281111EC08091BB008093E60203
:104E80008091E602823120F01092E60280E001C0BB
:104E900081E091E09093E5022091E60230E04091BC
:104EA0000601509107014217530709F090E09093D3
:104EB000E70246C0E091E602F0E08091BB00EF5AC5
:104EC000FC4F80838091E6028F5F8093E6028091A1
:104ED000E7028823A1F1C091C201D091C301A8814A
:104EE00088E0A802D0011124AB5FBE4F1696ED9169
:104EF000FC911797309719F114962D913C911597C5
:104F00002C0F3D1F11968D919C911297BE01680F39
:104F1000791F13964C9113978C91099510C0E091CD
:104F2000E602F0E0EF5AFC4F80818093BB00809155
:104F3000E6028F5F8093E60202C01092BC0081E01F
:104F40009091BC008295880F880F807C9568892B92
:104F50008093BC00FF91EF91DF91CF91BF91AF9112
:104F60009F918F917F916F915F914F913F912F9181
:104F70000F900FBE0F901F9018959093EB018093A8
:104F8000EA0108959093EE028093ED0208950E9445
:104F90003C15811103C08091E8020895E091ED0273
:104FA000F091EE02309721F00190F081E02D09940C
:104FB00080E00895E091ED02F091EE02309799F0D3
:104FC00020915401222359F020911A0327FF07C092
:104FD000DC012C9111962C93119726E02C930280E2
:104FE000F381E02D09940895E091ED02F091EE0235
:104FF000309739F022E0DC012C930480F581E02D1C
:10500000099408952091EB023091EC02281739079A
:1050100071F09093EC028093EB02E091ED02F0913D
:10502000EE02309721F00680F781E02D0994089573
:105030002091E9023091EA022817390771F0909324
:10504000EA028093E902E091ED02F091EE023097DE
:1050500021F00084F185E02D09940895FC01329639
:1050600080915401882331F080911A0387FF02C098
:105070009EE101C096E080E0915028F0219122232A
:10508000D9F38F5FF9CF0895662351F12091540130
:105090002223E9F020911A0327FF19C0462F4695D5
:1050A000469546954E31E0F4677021E030E002C04D
:1050B000220F331F6A95E2F7FC01E40FF11D828194
:1050C00090E02823392381E0232B69F409C0FC01F7
:1050D000329608962191621729F0E817F907D1F75F
:1050E00080E0089581E008959C01FC0132969FEFD5
:1050F00080E04191461789F09F3F19F4411101C0AA
:10510000982F8F5F8630A9F79F3F39F0F901E90F9B
:10511000F11D97FDFA956283089508959C012A5F19
:105120003F4FFC014281461301C012820196821753
:105130009307B9F70895262F2695269526952E31A3
:1051400068F4FC01E20FF11D677021E030E001C05E
:10515000220F6A95EAF78281282B22830895262F51
:105160002695269526952E3170F4FC01E20FF11D4F
:10517000677021E030E001C0220F6A95EAF72095C0
:10518000828128232283089520915401222329F02B
:1051900020911A0327FD0C949B280C9474282091CD
:1051A0005401222329F020911A0327FD0C94AF28E3
:1051B0000C948E2820915401FC013296222331F068
:1051C00080911A0387FF02C08EE101C086E0DF01F3
:1051D0001D928A95E9F7089508950C94EC2883E0D0
:1051E0008093EF020C94ED28811102C081E001C090
:1051F00082E08093EF020C94ED280C94F42881E077
:105200008093EF020C94ED280C94FF2808950C94E1
:1052100006290C9407290C9406290C9406290C9451
:105220000629CF930E940D290E94B1140E940B29D8
:10523000C0E08C2F0E947613811104C0CF5FC8306C
:10524000C1F701C081E0CF91089508951F920F9298
:105250000FB60F9211248F939F93AF93BF938091BA
:10526000F002811113C08091630390916403A091B7
:105270006503B09166034196A11DB11D8093630340
:1052800090936403A0936503B0936603BF91AF91BD
:105290009F918F910F900FBE0F901F901895809146
:1052A0006B03843031F10E94FB031092F00220E482
:1052B00088E190E00FB6F894A895809360000FBE47
:1052C0002093600083B7817F846083BF83B7816050
:1052D00083BF7894889583B78E7F83BF0FB6F89489
:1052E000A8958091600088618093600010926000B2
:1052F0000FBE08950E9425090C94010482E084BD2C
:1053000093E095BD9AEF97BD80936E0008952FB7F7
:10531000F8948091630390916403A0916503B09128
:1053200066032FBF08952FB7F894609163037091BF
:10533000640380916503909166032FBF08959C01DB
:105340004FB7F8948091630390916403A091650333
:10535000B09166034FBF821B930B0895CF92DF92EB
:10536000EF92FF922FB7F894C0906303D09064033C
:10537000E0906503F09066032FBFA7019601261BFE
:10538000370B480B590BCA01B901FF90EF90DF9022
:10539000CF90089578941F920F920FB60F92112418
:1053A0008F939F93AF93BF93809163039091640316
:1053B000A0916503B09166030196A11DB11D809374
:1053C000630390936403A0936503B0936603BF9156
:1053D000AF919F918F910F900FBE0F901F901895D6
:1053E00087E797E790930108809300089AE088E1A7
:1053F0000FB6F894A895809360000FBE909360005C
:10540000FFCF809114030895089522E02093E900CE
:105410002FEF3091E800215035FD06C035ED3A956B
:10542000F1F700002111F5CF2091E80025FF0BC016
:1054300040E050E066E070E00E94442C8091E8007B
:105440008E778093E8000895CF93DF9320915401E5
:10545000222339F020911A0327FF03C060E222E0E3
:1054600002C068E021E02093E9002FEF3091E800CE
:10547000215035FD06C035ED3A95F1F700002111B8
:10548000F5CF2091E80025FF1DC0EC01809154016B
:10549000811105C040E050E068E070E003C070E0BA
:1054A00040E050E0CE010E94442C8091E8008E77CD
:1054B0008093E80080E2FE01A4EFB2E001900D923B
:1054C0008A95E1F7DF91CF9108958093F10270936F
:1054D000F3026093F20280916B03843001F582E065
:1054E0008093E9008FEF9091E800815095FD06C010
:1054F00095ED9A95F1F700008111F5CF8091E800C4
:1055000085FF0DC040E050E063E070E081EF92E085
:105510000E94442C8091E8008E778093E8000895E3
:10552000BC0184E00C94652ABC0183E00C94652ADC
:1055300080916A03811109C00E94D52D0E94322EEC
:105540008091E20084608093E200089510926A03E3
:1055500008950C9404296091670381E0611101C0F2
:1055600080E00C94EF2890916B0381E0943009F077
:1055700080E0609167030C94F42842E061EC81E0E4
:105580000E944E2D42E261EC82E00E944E2D9091ED
:105590006B0381E0943009F080E0609167030C9424
:1055A000FD2880916D03833009F461C030F48130AF
:1055B00071F0823009F49AC008958A3009F486C0E7
:1055C0008B3009F46CC0893009F0A8C020C08091EC
:1055D0006C03813A09F0A2C08091E800877F809334
:1055E000E8008091700390917103892B21F460E2AF
:1055F00084EF92E003C060E080E090E070E00E9401
:105600008F2C8091E8008B778093E800089580913B
:105610006C03813209F082C0809170039091710314
:10562000029708F07BC08091E800877F8093E800B4
:105630008091E80082FD05C080916B038111F8CF55
:105640006DC02091F3008091F20090E0922B0297C0
:1056500031F48091F100813011F0863021F4809195
:10566000F100809314038091E8008B7753C0809100
:105670006C03813A09F052C08091700390917103DC
:10568000892B09F04BC08091E800877F8093E80068
:105690008091E80080FFFCCF8091540136C080915A
:1056A0006C038132D9F58091700390917103892B3D
:1056B000A9F58091E800877F8093E8000E94832D00
:1056C00080916E03809354010C94250980916C03A2
:1056D000813221F58091E800877F8093E8000E9465
:1056E000832D80916F0380931503089580916C033F
:1056F000813AA1F48091E800877F8093E80080914F
:10570000E80080FFFCCF809115038093F100809129
:10571000E8008E778093E8000C94832D089584B779
:10572000877F84BF0FB6F894A89580916000886148
:1057300080936000109260000FBE90E080E80FB68A
:10574000F89480936100909361000FBE0C94FF2841
:105750000E94D52D0E94322EE2EEF0E0808184601E
:10576000808378940C94C73088E491E00C94C2272D
:1057700080916B038530A9F480916B03853079F4B7
:105780000E944F29809169038823B1F30E94112957
:10579000882391F30E942E2C0E942509EDCF0C94B2
:1057A0007A29089508950C94D52B292F3327233077
:1057B0003105C9F060F42130310581F02230310526
:1057C00009F044C08BE390E021EE34E043C0213285
:1057D0003105E1F02232310549F138C082E190E033
:1057E0002CE135E037C099278130910549F028F048
:1057F000029761F5E9EBF4E005C0EDEDF4E002C0DD
:10580000E7ECF4E0849190E09F0124C061157105FC
:1058100041F061307105D1F489E090E02CE035E091
:1058200019C089E090E023EF34E014C061157105E0
:1058300041F06130710551F486EB90E02EE235E0E5
:1058400009C080E490E024EE35E004C080E090E000
:1058500020E030E0FA0131832083089580E189BDA2
:1058600082E189BD09B400FEFDCF8091D8008F7D13
:105870008093D8008091E00082608093E000809166
:10588000E00081FDFCCF0895CF92DF92EF92FF926E
:105890000F931F93CF93DF93EC018B017A010E944A
:1058A000A22D811133C0E114F10439F0F701808198
:1058B0009181081B190BC80FD91FC12CD12C0115C0
:1058C000110519F18091E80085FD16C08091E8006E
:1058D0008E778093E800E114F10449F0F7018081AC
:1058E0009181C80ED91ED182C08285E00FC00E946E
:1058F000A22D882321F30AC089918093F1000150E1
:105900001109FFEFCF1ADF0ADACF80E0DF91CF91E4
:105910001F910F91FF90EF90DF90CF90089520910D
:105920007203309173032617370748F0611571052C
:1059300039F42091E8002E772093E80001C0B901E6
:10594000FC0120E06115710579F180916B038823DA
:10595000F1F18530F1F18091E80083FD3CC0809148
:10596000E80082FD2EC08091E80080FFEBCF2091FF
:10597000F3008091F20090E0922B6115710551F0D7
:105980008830910538F421912093F100615071091C
:105990000196F3CF21E0089709F020E08091E8001C
:1059A0008E778093E800CECF2111CFCF0AC08091AF
:1059B0006B03882361F0853061F08091E80083FDFE
:1059C0000AC08091E80082FFF2CF80E0089582E073
:1059D000089583E0089581E0089520917203309145
:1059E00073032617370748F06115710539F42091C4
:1059F000E8002E772093E80001C0B901FC0120E007
:105A00006115710591F180916B03882309F440C001
:105A1000853009F43FC08091E80083FD3DC080914E
:105A2000E80082FD2FC08091E80080FFE9CF20913F
:105A3000F3008091F20090E0922B6115710559F00E
:105A40008830910540F424912093F1003196615003
:105A500071090196F2CF21E0089709F020E08091CA
:105A6000E8008E778093E800CBCF2111CCCF0AC01D
:105A700080916B03882361F0853061F08091E800AC
:105A800083FD0AC08091E80082FFF2CF80E0089594
:105A900082E0089583E0089581E00895982F97307B
:105AA00068F59093E900981739F07091EC00209117
:105AB000ED005091F00003C0242F762F50E021FD1F
:105AC00002C09F5FECCF3091EB003E7F3093EB0044
:105AD0003091ED003D7F3093ED003091EB0031606F
:105AE0003093EB007093EC002093ED005093F000A6
:105AF0002091EE0027FDE5CF80E008958F70809320
:105B0000E90081E0089580916C0387FF11C08091C6
:105B1000E80082FD05C080916B038111F8CF11C0B0
:105B20008091E8008B770BC080916B03882349F04C
:105B30008091E80080FFF8CF8091E8008E77809315
:105B4000E80008952091E4003091E50095E6409149
:105B5000EC00842F817040FF23C08091E80080FD1D
:105B60001DC080916B03882399F0853099F0809156
:105B7000EB0085FD11C04091E4005091E500241731
:105B8000350729F3915011F09A01E1CF84E008958F
:105B900082E0089583E0089581E0089580E008950B
:105BA0004091E80042FFDDCF08950E94432E0E94FD
:105BB0004B2EE0EEF0E0808181608083E8EDF0E044
:105BC00080818F77808319BCA7EDB0E08C918E7FA8
:105BD0008C9380818F7E808310926A0308950F9347
:105BE0001F93CF93DF930E94432E0E944B2EC8ED4C
:105BF000D0E088818F7788838881806888838881D6
:105C00008F7D888319BC10926B03109267031092EA
:105C100069031092680300EE10E0F80180818B7F29
:105C2000808388818160888342E060E080E00E9418
:105C30004E2DE1EEF0E080818E7F8083E2EEF0E099
:105C4000808181608083808188608083F801808189
:105C50008E7F8083888180618883DF91CF911F91BF
:105C60000F910895E8EDF0E080818F7E8083E7ED6D
:105C7000F0E080818160808384E082BF81E0809356
:105C80006A030C94EF2DE8EDF0E080818E7F808335
:105C90001092E20008951092DA001092E100089547
:105CA0001F920F920FB60F9211242F933F934F9391
:105CB0005F936F937F938F939F93AF93BF93EF9374
:105CC000FF938091E10082FF0BC08091E20082FF90
:105CD00007C08091E1008B7F8093E1000E94C63075
:105CE0008091DA0080FF1FC08091D80080FF1BC028
:105CF0008091DA008E7F8093DA008091D90080FF56
:105D00000DC080E189BD82E189BD09B400FEFDCFEF
:105D100081E080936B030E94982A05C019BC109201
:105D20006B030E94A62A8091E10080FF19C0809138
:105D3000E20080FF15C08091E2008E7F8093E20038
:105D40008091E20080618093E2008091D8008062BF
:105D50008093D80019BC85E080936B030E94AB2A26
:105D60008091E10084FF30C08091E20084FF2CC06C
:105D700080E189BD82E189BD09B400FEFDCF80913B
:105D8000D8008F7D8093D8008091E1008F7E809332
:105D9000E1008091E2008F7E8093E2008091E2003A
:105DA00081608093E20080916703882311F084E092
:105DB00007C08091E30087FD02C081E001C083E05D
:105DC00080936B030E94B32A8091E10083FF29C076
:105DD0008091E20083FF25C08091E100877F80935E
:105DE000E10082E080936B03109267038091E100F1
:105DF0008E7F8093E1008091E2008E7F8093E200AD
:105E00008091E20080618093E20042E060E080E007
:105E10000E944E2D8091F00088608093F0000E94D7
:105E2000A92AFF91EF91BF91AF919F918F917F919F
:105E30006F915F914F913F912F910F900FBE0F90F7
:105E40001F9018951F920F920FB60F9211242F9347
:105E50003F934F935F936F937F938F939F93AF93F2
:105E6000BF93CF93DF93EF93FF93C091E900CF707F
:105E70008091EC00D82FD17080FDD0E81092E9001D
:105E80008091F000877F8093F00078940E94662FC5
:105E90001092E9008091F00088608093F000CD2B93
:105EA000CF70C093E900FF91EF91DF91CF91BF9147
:105EB000AF919F918F917F916F915F914F913F91A2
:105EC0002F910F900FBE0F901F9018951F93CF9397
:105ED000DF93CDB7DEB7AA970FB6F894DEBF0FBE3B
:105EE000CDBFECE6F3E08091F100819323E0E4374D
:105EF000F207C9F70E94D12A8091E80083FF2EC1E2
:105F000080916C0390916D03492F50E04A30510508
:105F100008F024C1FA01EE59FF4F0C9495348038F3
:105F200021F0823809F01AC108C08091680390916D
:105F30006903992389F082600FC0809170038F708C
:105F4000873008F00BC18093E9008091EB0085FB5E
:105F5000882780F91092E9009091E800977F90934C
:105F6000E8008093F1001092F100D1C0282F2D7F1E
:105F700009F0F4C0882319F0823061F0EFC08091FD
:105F80006E03813009F0EAC0933009F080E080931D
:105F900069032EC080916E0381112AC08091700325
:105FA0008F702FEF280F263008F0D8C08093E900BB
:105FB0002091EB0020FF1CC0933021F48091EB0076
:105FC000806214C09091EB0090619093EB0021E00F
:105FD00030E0A90102C0440F551F8A95E2F74093B3
:105FE000EA001092EA008091EB0088608093EB0059
:105FF0001092E9008091E800877F8093E8000E947A
:10600000832DACC08111AAC010916E031F778091BF
:10601000E3008078812B8093E3008091E800877F04
:106020008093E8000E94832D8091E80080FFFCCFE0
:106030008091E30080688093E300111102C082E048
:1060400001C083E080936B0389C08058823008F0E0
:1060500085C080916E0390916F038C3D53E095074E
:1060600079F583E08A838AE289834FB7F894DE0169
:10607000139620E03EE051E2E32FF0E0509357000A
:10608000E49120FF03C0E295EF703F5FEF708E2F29
:1060900090E0EA3010F0C79601C0C0968D939D93B2
:1060A0002F5F243149F74FBF8091E800877F8093AD
:1060B000E8006AE270E0CE0101960E948F2C16C0C3
:1060C0006091700370917103AE014F5F5F4F0E944A
:1060D000D32BBC01892B09F441C09091E800977F34
:1060E0009093E80089819A810E94ED2C8091E800CC
:1060F0008B778093E80032C0803881F58091E8008A
:10610000877F8093E800809167038093F1008091FE
:10611000E8008E7772CF811121C080916E0390913B
:106120006F0399270297D4F48091E800877F8093CA
:10613000E80080916E03809367030E94832D809115
:106140006703811106C08091E30087FD02C081E0F2
:1061500001C084E080936B030E94BD2A8091E80017
:1061600083FF0AC08091E800877F8093E8008091D8
:10617000EB0080628093EB00AA960FB6F894DEBF26
:106180000FBECDBFDF91CF911F9108950895CF939A
:1061900080916B038823A1F0C091E900CF709091AA
:1061A000EC00892F817090FD80E8C82B1092E900E7
:1061B0008091E80083FD0E94662FCF70C093E900B4
:1061C000CF9108950E94D52D10926B030895E8EDAC
:1061D000F0E08081806180838AE18A95F1F700C0D8
:1061E0008091D900817008955058BB27AA270E943A
:1061F0000C310C94B7320E94A93238F00E94B032B0
:1062000020F039F49F3F19F426F40C947F320EF4F9
:10621000E095E7FB0C947932E92F0E94C83258F3DD
:10622000BA17620773078407950720F079F4A6F57B
:106230000C94EA320EF4E0950B2EBA2FA02D0B0130
:10624000B90190010C01CA01A0011124FF27591BBB
:1062500099F0593F50F4503E68F11A16F040A22FC1
:10626000232F342F4427585FF3CF46953795279532
:10627000A795F0405395C9F77EF41F16BA0B620B31
:10628000730B840BBAF09150A1F0FF0FBB1F661F78
:10629000771F881FC2F70EC0BA0F621F731F841FBB
:1062A00048F4879577956795B795F7959E3F08F0E1
:1062B000B0CF9395880F08F09927EE0F97958795A3
:1062C00008950E9475310C94B7320E94B03258F094
:1062D0000E94A93240F029F45F3F29F00C947932F2
:1062E00051110C94EB320C947F320E94C83268F347
:1062F0009923B1F3552391F3951B550BBB27AA277F
:1063000062177307840738F09F5F5F4F220F331FB8
:10631000441FAA1FA9F335D00E2E3AF0E0E832D080
:1063200091505040E695001CCAF72BD0FE2F29D083
:10633000660F771F881FBB1F261737074807AB0755
:10634000B0E809F0BB0B802DBF01FF2793585F4FCA
:106350003AF09E3F510578F00C9479320C94EB3270
:106360005F3FE4F3983ED4F3869577956795B795AC
:10637000F7959F5FC9F7880F911D9695879597F9B7
:106380000895E1E0660F771F881FBB1F6217730730
:106390008407BA0720F0621B730B840BBA0BEE1F45
:1063A00088F7E095089529F416F00C9479320C944E
:1063B000EA320C947F320E94D032A8F39638A0F7CC
:1063C00007F80F92E8942BE33AEA48EB5FE70E9464
:1063D0007D330F920F920F924DB75EB70F920E94CE
:1063E0003333E8EDF0E00E9482324F915F91EF91FC
:1063F000FF91E595EE1FFF1F49F0FE57E068442727
:10640000EE0F441FFA95E1F74195550B0E94FD32BE
:106410000F9007FE0C94F13208950E94D03288F05C
:106420009F5798F0B92F9927B751B0F0E1F0660F58
:10643000771F881F991F1AF0BA95C9F714C0B13099
:1064400091F00E94EA32B1E008950C94EA32672F8D
:10645000782F8827B85F39F0B93FCCF386957795C8
:106460006795B395D9F73EF49095809570956195B1
:106470007F4F8F4F9F4F0895E89409C097FB3EF4DC
:1064800090958095709561957F4F8F4F9F4F992381
:10649000A9F0F92F96E9BB279395F69587957795FF
:1064A0006795B795F111F8CFFAF4BB0F11F460FFBF
:1064B0001BC06F5F7F4F8F4F9F4F16C0882311F017
:1064C00096E911C0772321F09EE8872F762F05C02B
:1064D000662371F096E8862F70E060E02AF09A95C6
:1064E000660F771F881FDAF7880F9695879597F9BB
:1064F000089597F99F6780E870E060E008959FEF46
:1065000080EC0895DF93CF931F930F93FF92EF9248
:10651000DF927B018C01689406C0DA2EEF010E94A5
:106520007A33FE01E894A5912591359145915591D5
:10653000A6F3EF010E940C31FE019701A801DA9445
:1065400069F7DF90EF90FF900F911F91CF91DF914E
:10655000089500240A9416161706180609060895C9
:1065600000240A9412161306140605060895092E2F
:106570000394000C11F4882352F0BB0F40F4BF2B9E
:1065800011F460FF04C06F5F7F4F8F4F9F4F0895DE
:1065900057FD9058440F551F59F05F3F71F04795D4
:1065A000880F97FB991F61F09F3F79F087950895B9
:1065B000121613061406551FF2CF4695F1DF08C0D8
:1065C000161617061806991FF1CF869571056105F5
:1065D00008940895E894BB2766277727CB0197F99D
:1065E00008959B01AC0160E070E080E89FE30C94AB
:1065F00061310C9479320C94DC330E94D032D8F3A0
:106600009923C9F3940F511DA3F39150504094F076
:1066100059F0882332F0660F771F881F9150504041
:10662000C1F79E3F51052CF7880F911D96958795D0
:1066300097F908955F3FACF0983E9CF0BB27869594
:1066400077956795B79508F4B1609395C1F7BB0F3F
:1066500058F711F460FFE8CF6F5F7F4F8F4F9F4F68
:10666000E3CF0C94EB32FA01DC01AA0FBB1F9B01B4
:10667000AC01BF5728F4222733274427507820C085
:10668000B75190F4AB2F0024469537952795011C00
:10669000A395D2F3002071F0220F331F441FB3954E
:1066A000DAF30ED00C94F43061307105A0E88A075B
:1066B000B94630F49B01AC0166277727882790788C
:1066C000309621F0208331834283538308950E94C2
:1066D0007A330C94B7320E94A93238F00E94B0325B
:1066E00020F0952311F00C9479320C947F32112410
:1066F0000C94EB320E94C83270F3959FC1F3950F52
:1067000050E0551F629FF001729FBB27F00DB11D35
:10671000639FAA27F00DB11DAA1F649F6627B00DC5
:10672000A11D661F829F2227B00DA11D621F739FAE
:10673000B00DA11D621F839FA00D611D221F749FBC
:106740003327A00D611D231F849F600D211D822F03
:10675000762F6A2F11249F5750409AF0F1F088232A
:106760004AF0EE0FFF1FBB1F661F771F881F915057
:106770005040A9F79E3F510580F00C9479320C945B
:10678000EB325F3FE4F3983ED4F3869577956795B7
:10679000B795F795E7959F5FC1F7FE2B880F911D81
:1067A0009695879597F908959F930E94EC330F90E3
:1067B00007FCEE5F0C9415349F3F31F0915020F4AC
:1067C000879577956795B795880F911D96958795CD
:1067D00097F908950C947F320E94D032D8F3E89450
:1067E000E0E0BB279F57F0F02AED3FE049EC06C000
:1067F000EE0FBB0F661F771F881F28F0B23A6207A3
:106800007307840728F0B25A620B730B840BE3956D
:106810009A9572F7803830F49A95BB0F661F771FF0
:10682000881FD2F790480C94DE33EF93E0FF07C047
:10683000A2EA2AED3FE049EC5FEB0E940C310E9496
:10684000B7320F90039401FC9058E0E0F1E00C9413
:1068500029349F938F937F936F93FF93EF939B01C3
:10686000AC010E946733EF91FF910E9482322F9119
:106870003F914F915F910C94673387FB082E06265A
:1068800087FD819567FD61950E94CC340EF491954A
:1068900007FC81950895AA1BBB1B51E107C0AA1FE5
:1068A000BB1FA617B70710F0A61BB70B881F991FB1
:1068B0005A95A9F780959095BC01CD01089597FB55
:1068C000072E16F4009407D077FD09D00E944B34B0
:1068D00007FC05D03EF4909581959F4F08957095E3
:1068E00061957F4F0895A1E21A2EAA1BBB1BFD01E3
:1068F0000DC0AA1FBB1FEE1FFF1FA217B307E4079F
:10690000F50720F0A21BB30BE40BF50B661F771FF6
:10691000881F991F1A9469F76095709580959095D6
:106920009B01AC01BD01CF010895EE0FFF1F059043
:10693000F491E02D09940E94A334332312F48A1BAE
:106940009B0B0C94B434A29FB001B39FC001A39FD2
:10695000700D811D1124911DB29F700D811D112498
:10696000911D08950E94A334B7FF0895821B930BD5
:1069700008950E94A334A59F900DB49F900DA49FED
:10698000800D911D11240895B7FF0C94B9340E9415
:10699000B934821B930B0895991B79E004C0991FA9
:1069A000961708F0961B881F7A95C9F78095089569
:1069B000FC014150504030F001900616D1F731975C
:1069C000CF010895882799270895FB01DC0104C0B1
:1069D0008D910190801921F441505040C8F7881BD7
:1069E000990B0895FB01DC0102C001900D9241500A
:1069F0005040D8F70895F999FECF92BD81BDF89A1D
:106A0000992780B50895A6E1B0E044E050E00C94E9
:106A10003535A8E1B0E042E050E00C943535262F42
:106A2000F999FECF92BD81BDF89A019700B4021684
:106A300039F01FBA20BD0FB6F894FA9AF99A0FBE32
:106A400008950396272F0E9410350E940F35252F99
:106A50000E941035242F0C9410350196272F0E9488
:106A600010350C940F35DC01CB01FC01F999FECFF8
:106A700006C0F2BDE1BDF89A319600B40D924150C6
:0A6A80005040B8F70895F894FFCFD6
:106A8A00C8007302010100000000000000000000BD
:106A9A0001010000000000000402000000040600DA
:106AAA000000000000080A0000000000002808504A
:106ABA00011E0A1401010102000A000A0A01191A38
:106ACA001B1C1D1E1F202122012A242A052A942A62
:106ADA00902A042A01E200E900EA00B500B600B7EC
:106AEA0000CD008301CC008A019201940121022386
:106AFA000224022502260227022A02B300B4006FEA
:106B0A00007000818283E200E900EA00B500B60065
:106B1A00B700CD008301CC008A01920194012102C1
:106B2A00230224022502260227022A02B300B40005
:106B3A006F0070008182839497C6333236F4F76609
:106B4A00F6F55103000102020202060606090909C6
:106B5A000909090F0F0F0F0F0F1515151819191914
:0A6B6A00191919191919192324002B
:00000001FF
